:020000040800F2
:10000000D809002001030008090300080B030008B9
:100010000D0300080F030008110300080000000092
:10002000000000000000000000000000390200088D
:100030001503000800000000B1020008ED020008EE
:100040001B0300081B0300081B0300081B03000818
:100050001B0300081B0300081B0300081B03000808
:100060001B0300081B0300081B0300081B030008F8
:100070001B0300081B0300081B0300081B030008E8
:100080001B0300081B0300081B0300081B030008D8
:100090001B0300081B0300081B0300081B030008C8
:1000A0001B0300081B0300081B0300081B030008B8
:1000B000E95500081B0300081B0300081B03000888
:1000C0001B0300081B0300081B0300081B03000898
:1000D0001B030008A95600081B0300081B030008A7
:1000E0001B0300081B0300081B03000800F002F8B4
:1000F00000F04DF80AA090E8000C82448344AAF175
:100100000107DA4501D100F042F8AFF2090EBAE872
:100110000F0013F0010F18BFFB1A43F0010318473B
:10012000547D0000747D0000103A24BF78C878C167
:10013000FAD8520724BF30C830C144BF04680C60ED
:10014000704700000023002400250026103A28BF35
:1001500078C1FBD8520728BF30C148BF0B60704739
:10016000662907F06485642900F05281732900F044
:100170004E85002070471FB500F04DFD04000020A3
:10018000002106F0D1FFE0601FBD10B510BD00F0EA
:1001900045FE1146FFF7EFFF0FB400F00BF80FBC60
:1001A00005F058FD00F00CFA03B4FFF7EEFF03BCB6
:1001B00000F02EFE04B005F027FE0448002105F0F3
:1001C000D3FE05F033FE00F0FBF90000BC7D000813
:1001D00080F309887047EFF309807047684680F321
:1001E000098804480078C00714BF0220032080F368
:1001F000148870477C7D0008DFF818C0EFF3058392
:100200001B0618BF6047EFF31483DB0708BF604786
:1002100000DF704755600008DFF818C0EFF3058372
:100220001B0618BF6047EFF31483DB0708BF604766
:1002300000DF704739620008EFF30980816911F827
:10024000021CF1B990E80F10E047EFF3098C8CE83D
:100250000700144B93E8060091420FD039B12CE906
:10026000F00FC1F828C00CB406F06CFB0CBC1A608F
:10027000D2F828C0BCE8F00F8CF309886FF0020EAA
:10028000704710B5084A1268914209D8074C54F8D3
:10029000214090E80F10A047EFF3098C8CE80F0085
:1002A00010BD0000F0000020F8150008F815000847
:1002B00006F0DEF90C4B93E80600914210D0EFF304
:1002C000098C2CE9F00FC1F828C00CB406F03AFBF9
:1002D0000CBC1A60D2F828C0BCE8F00F8CF3098877
:1002E0006FF0020E70470000F000002006F0F2FBF5
:1002F000E0E7000005F09AFE06F0ECFBDAE700000C
:100300000948804709480047FEE7FEE7FEE7FEE7A9
:10031000FEE7FEE7FEE7FEE7FEE7FEE704480549E5
:10032000054A064B7047000089550008ED0000089B
:10033000D8030020D8090020D8050020D8050020C7
:1003400000487047780300200FB41CB5074B06AA7D
:100350007B4469460090059800F02FFC0020694618
:1003600000F03EFC1CBC5DF814FB00008D08000092
:1003700070B5044685690068C10601D5302600E0E5
:100380002026C00707D070BDD4E901213046904730
:10039000206A401C20626D1EF6D570BD70B5044603
:1003A00085690078C00707D170BDD4E901212020FC
:1003B0009047206A401C20626D1EF6D570BD70B556
:1003C0000C460546012A05D02878800600D5EA6942
:1003D000002302E0012305E05B1C934202D2E05CB3
:1003E0000028F9D1A869E618C01AA861286A18443B
:1003F00028622846FFF7BCFF04E0D5E9012114F884
:10040000010B9047B442F8D32846FFF7C7FF70BDF1
:100410002DE9F0410646002410687529314616A5DD
:1004200010D0AFF30080002802DA404213A507E0A5
:1004300031688A0701D512A502E0490704D511A544
:10044000012401E0AFF3008000210A2206F1240715
:1004500009E0B0FBF2FCB0FBF2F302FB1C00303011
:1004600078541846491C0028F3D123462A463046C2
:10047000BDE8F04100F033B9000000002D0000009D
:100480002B000000200000002DE9F05F89460446A3
:100490004FF0000ADFF824B1FB44C0F820A020464A
:1004A000E168884700287DD0252806D0D4E90121BD
:1004B0009047206A401C2062F1E700255F462046F5
:1004C000E16888472028064607DB312E05D2B81997
:1004D00010F8200C08B10543F1E7A80701D525F075
:1004E0000405C4F81CA00027C4F818A02A2E09D0BF
:1004F000304605F059FA38B304EB8708303EC8F8A7
:10050000186019E059F8041B204604EB870291613A
:10051000E1688847012F064618D1E069002820DAF3
:1005200025F020051DE0D8F8180000EB800006EB50
:1005300040003038C8F818002046E1688847064671
:1005400005F032FA0028EED1012F0AD02E2E08D164
:100550002046E16888477F1C0646022F45F02005AB
:10056000C4DBA069002803DA404245F00105A06120
:10057000E80701D025F01005A6B1A6F14100192821
:1005800002D8203645F400654A46314620462560AB
:100590004D46FFF7E5FD60B1012807D0ED1D25F0C0
:1005A000070000E007E000F1080978E705F1040919
:1005B00075E730467AE7206ABDE8F09F30790000A1
:1005C00010B50446AFF300802046BDE81040FFF7A9
:1005D000EBBD40EA0103024630B59B0710D14FF056
:1005E000013400E008C208C91D1B9D4315EAC41F61
:1005F000F8D013F0FF0102F8011B0DD01B0AF8E739
:1006000011F8013B002B02F8013B05D011F8013B2A
:10061000002B02F8013BF3D130BD10B5431C02E0C2
:1006200010F8011B71B18107FAD14FF0013202C8F5
:100630008C1A8C4314EAC211F9D0C01A0A0603D0EE
:10064000C01E10BDC01A10BD0A0401D0801E10BD0E
:100650000902FCD0401E10BD4FF0013C50F8042BA5
:1006600051F8043B9A4221D1A2EB0C03934313EAC5
:10067000CC1317D150F8042B51F8043B9A4215D1F2
:10068000A2EB0C03934313EACC130BD150F8042BC9
:1006900051F8043B9A4209D1A2EB0C03934313EAAD
:1006A000CC13DBD04FF00000704700BFD01A01BA66
:1006B000B1FA81F101F0180122FA01F0CB40C1F149
:1006C0002001DBB2C0B2C01A2CFA01F3D11A914357
:1006D00011EAC311E6D170477047704770472DE9A2
:1006E000F0470D4699469246044600F124080168F9
:1006F000880604D5E06921F01001216000E00120A6
:10070000A84201DD471B00E00027A1697A1902EB2E
:100710000900081AA0612078C00602D42046FFF71D
:1007200027FE002608E0D4E901211AF806009047C8
:10073000206A401C761C20624E45F4DB2078C006FF
:100740000AD52046FFF714FE06E0D4E90121302047
:100750009047206A401C2062381EA7F10107F4DC94
:1007600007E0D4E9012118F805009047206A401CF1
:100770002062281EA5F10105F3DC2046FFF70EFEDE
:100780002078000602D50220BDE8F0870120FBE7B3
:1007900070472DE9FF4F0C461E464FF0FF378BB0D8
:1007A000D2E90001DDF860800A908A46C1F30A555B
:1007B00005B93D46002108464FF00000BAF1000F90
:1007C00000F4400005DA00EB80004FF4400101EA3C
:1007D00050004FEA9059B9F1010F00DDB9460A986F
:1007E00050EA4A000ED044F61050A5F2FF354543BA
:1007F0002F14B8F1000F1ED07542291E1EDDC9F15D
:1008000000021CE0B8F1010F4FF0000001D03021D0
:1008100003E0F24305E02154401CB042FBDB3046CC
:100820000022002121540B99C1F80880C1E9002061
:100830000FB0BDE8F08FBD1B6D1CDEE74A4600DA45
:10084000694206A800F072FA06AB93E8070003AB12
:1008500083E8070050460A9900F006FB8DE8070080
:10086000A0F500501F3800900398002D0ADD42F2D9
:100870001F014A460844002303A90390684600F07C
:100880006FFD09E0A0F500504A461F38002303A978
:100890000390684600F079FD8DE807000004000C25
:1008A00003D04FF0FF30410800E01046B8F1000FD0
:1008B00003D00022009215461EE0751E05D400F0FC
:1008C000AFF9303262556D1EF9D5B34601220843A7
:1008D00002D000227F1C04E02078302801D10022C1
:1008E0007F1E002A099784D01DE0112D07DA00F041
:1008F00097F9303262556D1C50EA0102F5D1084378
:1009000002D00098C8B10EE00021681E05E0235C0B
:10091000625C63542254401E491C8142F7DBAB46A3
:10092000A81B401E0990002004F80B000B98099AA0
:10093000C0F80880C0E9002B7AE711264FF00008C4
:1009400057E72DE9F04F88460446D21D22F00701F3
:1009500091B0D1E90001CDE90A0104F0DDFF0246C2
:100960000B98C00F01D02D2007E02068810701D52A
:100970002B2002E0202101EAC000032A099001D0C7
:10098000072A05DB03464146204600F08FF90BE1BC
:100990002078800601D5E06900E00620B8F1650FF7
:1009A000814606D0B8F1660F18D0B8F1670F70D144
:1009B00031E00020B9F1110F009001DB112301E0BB
:1009C00009F101030AAA01A90CA8FFF7E2FEDDE97B
:1009D0000C70002609F10105834647E001204B46D3
:1009E00000904FF000470AAA01A90CA8FFF7D1FE1A
:1009F000DDE90DB00C995D46002610B909F1010042
:100A00000D18B9EB050003D4C0F1FF3609F101055B
:100A1000A5EB09002BE0B9F1010F01DA4FF0010954
:100A20000020B9F1110F0090484601DD112300E0CC
:100A300003460AAA01A90CA8FFF7ABFEDDE90C707A
:100A40004D4600268346207800070AD4AB4500DADD
:100A50005D4601A8012D04DD411911F8011C302962
:100A600007D04F4502DA17F1040F04DA012082465D
:100A70000FE06D1EEEE7002F02DCED1B3E4403E0AD
:100A8000781CA84200DD7D1CB81B00F1010A4FF064
:100A900000472078000703D4AA4501DB4FF0FF3A56
:100AA0000021B7F1004F0DF143088DF8431024D019
:100AB00002202B23002F01DA7F422D230A21021E60
:100AC000A0F1010000DC5FB197FBF1FC97FBF1F2B4
:100AD00001FB1C7C17460CF1300C08F801CDEEE749
:100AE000A8F1010003702188090501D5452100E026
:100AF0006521A0F1010800F8011C09980FA9A1EBDC
:100B00000807FF1D00B10120411901EBEA70A1693E
:100B10003844081A401EA0612078C00602D420463E
:100B2000FFF726FC099828B1D4E901219047206AF3
:100B3000401C20622078C00622D52046FFF718FC12
:100B40001EE0002E04DBB34502DD01A8805D00E05D
:100B50003020D4E901219047206A401C2062761C95
:100B6000AAF101005FEA000A0AD100F054F8C06857
:100B70000168405CD4E901219047206A401C206252
:100B8000281EA5F10105DCDC07E0D4E9012118F8F5
:100B9000010B9047206A401C2062381EA7F1010714
:100BA000F3DC2046FFF7FAFB032011B041E600001A
:100BB00001694A1C02610878704700B58FB0CDE921
:100BC00001310021059105497944CDE90310114611
:100BD0006846FFF759FC0FB000BD0000E5FFFFFFBE
:100BE0000A6802F8010B0A60704710B5436913B137
:100BF000AFF3008001E0FFF7E2FB012010BD1278A7
:100C000000F124010A7000224A700122EDE7116808
:100C10004FF0FF32E9E710B5FFF792FB203010BD2F
:100C200030B5B0F10A024FEA900E71F100034EEABE
:100C3000817EB0EB0E0061EB91014FEA101E4EEA8F
:100C4000017E10EB0E0041EB11114FEA102E4EEA1F
:100C5000016E10EB0E0041EB11214FEA104E4EEAEF
:100C6000014E10EB0E0041EB1141401841F1000123
:100C70004FEAD00040EA41704FEAD10110EB800505
:100C80004FEA810444EA907444EB01046D1944EB8B
:100C90000404521BA3414FF0000348BF0A3200D5A1
:100CA00030BD401C41F1000130BD00002DE9F04194
:100CB0001F46044603260168072A01F4006004DB8E
:100CC00008B116A505E016A503E008B115A500E0DA
:100CD00015A521F010002060A069C01EA0610FB111
:100CE000401EA0612046FFF743FB4FB1D4E901212C
:100CF00038469047206A401C2062C01C206206E0F3
:100D0000206AFAE7D4E9012115F8010B9047761E15
:100D1000F8D22046FFF742FBBDE8F0814E414E007D
:100D20006E616E00494E4600696E66002DE9F0471F
:100D3000814616468AB0354878440DC88DE80D00C6
:100D400032487844801C03AC0DC884E80D0041F69D
:100D50009B300844372190FBF1F290FBF1F5A5F1AF
:100D6000800501FB12041B3C02D56442012000E017
:100D70000020DFF898A080460027FA44AAF1BE0AB6
:100D80000EE0E0070AD03246684607EB4701012330
:100D90000AEB810100F0F9FA8DE8070064107F1C6E
:100DA000002CEED1194F7F44AE3F19E0E80715D073
:100DB00007EB04100DF1180A90E80E008AE80E0007
:100DC000C068F04201D1981908903246012306A963
:100DD00003A800F0DAFA03AB83E807006D10641C87
:100DE000002DE3D14FF0010332466946B8F1000F00
:100DF00003A802D000F0B4FA01E000F0C6FAC9E995
:100E00000001C9F808200AB0BDE8F0872071000091
:100E100001491820ABBEFEE7260002007546FFF729
:100E20008FFAAE4605006946534620F00700854616
:100E300018B020B5FFF772FABDE820404FF0000669
:100E40004FF000074FF000084FF0000B21F00701B2
:100E5000AC46ACE8C009ACE8C009ACE8C009ACE8F5
:100E6000C0098D46704770475FEA400C08BF91F09B
:100E7000000F4FEA8C234FEAC12243EA51514FEA57
:100E80001C5018BF00F5F0404FEA300018BF41F089
:100E900000415FEA6C5C00F02980BCF1FF3F08BFB5
:100EA00040F080407047130C06BF12044FF0100C46
:100EB0004FF0000C130E04BF12020CF1080C130FBC
:100EC00004BF12010CF1040C930F04BF92000CF14B
:100ED000020CD30F04BF52000CF1010C11464FF06D
:100EE0000002A0F11F00A0EB0C00704711F0004FB2
:100EF00008BF704731F000413FF4D5AF0B0C06BF7F
:100F000009044FF0100C4FF0000C0B0E04BF090247
:100F10000CF1080C0B0F04BF09010CF1040C8B0F32
:100F200004BF89000CF1020CCB0F04BF49000CF187
:100F3000010CCCF12003A0EB0C0022FA03F302FA1F
:100F40000CF241EA030100F10100704720F07F4CF0
:100F500080EA030023F07F47ACEB070303F57C53E3
:100F600000F0004003F1FF032DE980494FEA154BE3
:100F700009B44FEA144325EA0B4E24EA03480FF262
:100F8000042606EB132749083E785FEA320203FB8A
:100F90000667C7F5000707FB06F64FEA54374FEA26
:100FA000D64606F1020607FB066CCCF1005C4FEA60
:100FB0001C472CEA074C07FB06F40CFB06F504EB78
:100FC00015464FEA961634BF00204FF000404FEA16
:100FD000D13706FB07FC4FEA1C4C0CFB0BF7D21B6E
:100FE00003FB0CF761EB07010CFB0EF7B0EB0740BE
:100FF00072EB17420CFB08F734BFA2EB0742B2EBCF
:10100000074261EB17414FEA0C444FEA910706FB98
:1010100007FC4FEA1C4C0CFB0BF7B0EBC74072EB24
:10102000573203FB0CF734BFA2EBC742B2EBC74207
:1010300061EB57310CFB0EF7B0EBC70072EB577248
:101040000CFB08F734BFA2EBC702B2EBC70261EB9F
:101050005771039F4FEA816141EA921104EBCC047E
:101060004FEAD1374FEA826206FB07FC42EA901250
:101070004FEA80604FEA1C4C0CFB0BF7D21B03FBC2
:101080000CF761EB07010CFB0EF7B0EB074072EBBE
:1010900017420CFB08F734BFA2EB0742B2EB074242
:1010A00061EB17414FEA8C554FEA910704EB9C2402
:1010B00006FB07FC4FEA1C4C0CFB0BF7B0EBC740E0
:1010C00072EB573203FB0CF734BFA2EBC742B2EB13
:1010D000C74261EB57310CFB0EF7B0EBC70072EB68
:1010E00057720CFB08F734BFA2EBC702B2EBC70282
:1010F00061EB577115EB4C254FEA816141EA921182
:101100004FEA82624FEAD13742EA901206FB07FCAF
:1011100044F100044FEA80604FEA1C4C0CFB0BF7D3
:10112000D21B03FB0CF761EB07010CFB0EF7B0EBD6
:10113000074072EB17420CFB08F734BFA2EB0742E3
:10114000B2EB074261EB174115EB1C154FEA8131F9
:1011500041EA92414FEA823242EA90424FEA8030BD
:101160004FEA0C7644F1000448EA03434EEA0B4888
:101170004FF0000EB2EB080C71EB030724BF624680
:1011800039464EEB0E0E4FF0000B0018524149410C
:101190004BEB0B0BB2EB080C71EB03077BF1000B75
:1011A00024BF624639464EEB0E0E4FF0000B00187E
:1011B000524149414BEB0B0BB2EB080C71EB0307AF
:1011C0007BF1000B24BF624639464EEB0E0E51EA0E
:1011D000020718BF46F0010616EB0E7655F1000225
:1011E00054F1000103D5BDE88901BDE80088BDE8E0
:1011F0008901BDE80048B619524141EB0101A3F154
:101200000103704780807F7E7D7C7B7A797877765A
:1012100076757473727171706F6E6E6D6C6C6B6AD3
:101220006A69686867666665646463636261616071
:10123000605F5F5E5E5D5D5C5C5B5B5A5A595958EE
:101240005857575656555555545453535252525158
:10125000515050504F4F4F4E4E4D4D4D4C4C4C4BAE
:101260004B4B4A4A4A4949494848484747474746F5
:101270004646454545444444444343434342424231
:1012800042414141002B9C4630D477002BD01CB505
:101290004FEA370703B44FF010004FF01001BAF1D6
:1012A000000F06D0BCF1000FDCBF40F0080040F09A
:1012B00008014FF000000FBCBDE810400BF1010B1E
:1012C000BBF1010F08BF5FEA170722BF12F101024D
:1012D00011F101014FF0004143F1000300F0004023
:1012E00043EA00007047F9D35708D0E746EA0646BC
:1012F00013F1400F4FEA16461FDD13F1200FDFBF39
:1013000016430A46002120335B42BED0C3F12007BA
:1013100046EA064602FA07F74FEA164646EA070685
:10132000C3F1200722FA03F201FA07F721FA03F1C9
:101330004FF0000342EA0702A7E746EA020646EA40
:1013400006464FEA164646EA0106BCBF46EA06468E
:10135000360C4FF000034FF000024FF0000194E70D
:101360002DE9804C9A46934670B491E8380007C83E
:1013700031EA400C48BF34EA430C03D5FFF7E6FDE1
:10138000FFF780FFF0BCBDE8008C2DE9804C9A4649
:10139000934670B491E8380007C810F0804F08BF3A
:1013A00013F0804F03D100F005F8FFF76BFFF0BC9E
:1013B000BDE8008C20F07F4780EA030023F07F4CDB
:1013C00007EB0C03A3F57C5300F00040A3F1FE03F0
:1013D00092F0000F00F0B38095F0000F00F07780DE
:1013E0002DE901494FEA11404FEA144621EA00482D
:1013F00000FB06FC24EA064708FB06F607FB08F894
:1014000000FB07F718EB06484CEB164C4FEA124B63
:1014100018EB07484FEA15464CEB174022EA0B4EF3
:101420000BFB06FC25EA06470EFB06F607FB0EFE45
:101430000BFB07F71EEB064E4CEB164C4FF000066D
:101440001EEB074E4CEB174B18EB0B0840F100005E
:1014500018EB0E0B58EB000840F100008F1A4FF00C
:1014600000013CBFC943661B14BFB5EB040C00214F
:101470003CBFC943F61B4FEA17444EEA8E0E27EADB
:1014800004454FEA1C4704FB07622CEA074C05FBA6
:1014900007F70CFB05F604FB0CFC16EB074642EBCA
:1014A000174216EB0C4642EB1C421BEB060658EBB0
:1014B0000202414146EA9E0601D5BDE80189B619FE
:1014C000524141EB0101A3F10103BDE801894FEA5B
:1014D00014454FEA114724EA054621EA074C05FB6B
:1014E00007F406FB07F70CFB06F105FB0CFC11EB00
:1014F000074144EB17444FEA124711EB0C4144EB10
:101500001C4422EA074C05FB07F206FB07F70CFB1D
:1015100006F605FB0CFC16EB074642EB174216EBF2
:101520000C4642EB1C456A1854F1000148BF704755
:10153000B619524141EB0101A3F10103704795F047
:10154000000F37D04FEA11424FEA144721EA024612
:1015500024EA074C02FB07F106FB07F70CFB06F435
:1015600002FB0CFC14EB074441EB17414FEA154713
:1015700014EB0C4441EB1C4125EA074C02FB07F538
:1015800006FB07F70CFB06F602FB0CFC16EB074606
:1015900045EB174516EB0C4645EB1C42121951F171
:1015A000000148BF7047B619524141EB0101A3F158
:1015B000010370474FEA14454FEA114724EA0546F4
:1015C00021EA074C05FB07F106FB07F70CFB06F2C7
:1015D0004FF0000605FB0CFC12EB074241EB1741F4
:1015E00012EB0C4251EB1C4148BF7047921841EB83
:1015F0000101A3F1010370470000000010B504468B
:101600002CB94FF40041054802F0B9F904E04FF459
:101610000041024802F0B5F910BD00000008014089
:101620002DE9F041044600250A2C00DA12E040F2D0
:10163000DE30844201DD01250CE0204606F032F95F
:101640000746074906F076F9064606F0F3F8C0F1BA
:101650007F00C5B2284604F0CDF82046BDE8F081F1
:101660006F12033E10B50021014804F07DFC10BD4F
:10167000447C000870B503F06FFEFF2003F0AEFE5F
:10168000FF2003F0ABFEFF2003F0A8FEFF2003F0D5
:10169000A5FEFF2003F0A2FE322004F0A9FB2820C3
:1016A00000F00BF9054645F040052946282000F0DA
:1016B000BDFB052004F09CFB40F21F1631461020B4
:1016C00000F0A2FB052004F093FB40F2FF3004433E
:1016D0002146082000F098FB052004F089FB082033
:1016E00000F0D4F8044624F4600444F400042146D5
:1016F000082000F089FB052004F07AFB114800F077
:101700006BFB24F4600444F420042146082000F01C
:101710007BFB052004F06CFB0A4800F05DFB0A4CE3
:101720002146082000F070FB4FF080410748084A2E
:10173000C2E900100748114688600021064804F0FD
:1017400013FC70BD40420F00FF0308008171153F7C
:1017500028010020D65F0B00347C00082DE9F04101
:1017600000254CF2503000F037FB80B1182000F01B
:101770008DF805464148854205D941480078401C0E
:101780003F49087008E000203D49087004E03C48EB
:101790000078401C3A490870394800780A2869DD09
:1017A00003F0DAFDFF2003F019FEFF2003F016FE20
:1017B000FF2003F013FEFF2003F010FEFF2003F0D4
:1017C0000DFE322004F014FB282000F076F80646C7
:1017D00046F040063146282000F028FB052004F0A2
:1017E00007FB40F21F173946102000F00DFB0520C3
:1017F00004F0FEFA40F2FF3004432146082000F0D6
:1018000003FB052004F0F4FA082000F03FF804463A
:1018100024F4600444F400042146082000F0F4FAA3
:10182000052004F0E5FA174800F0D6FA24F4600425
:1018300044F420042146082000F0E6FA052004F0D4
:10184000D7FA104800F0C8FA0F4C2146082000F0E3
:10185000DBFA00200A4908704FF4FA7004F0C8FA65
:101860004CF2503000F0B8FA18B1182000F00EF821
:10187000054600BF2846BDE8F0810000C0E1E40055
:101880000000002040420F00FF03080070B505462D
:10189000002445F0400003F0A1FDFF2003F09EFD71
:1018A0000446FF2003F09AFD00EB0424FF2003F020
:1018B00095FD00EB0424204670BD70B5044600255C
:1018C00044F0400003F08AFDFF2003F087FD054649
:1018D000284670BD88B04FF4167004F089FAFFF7FF
:1018E0003DFFFE490860C82004F082FAFFF736FF8A
:1018F000FA4908600846006805F0BCFFF849074649
:10190000086005F07BFFF7490860F448006805F0BF
:10191000B1FF0746F448F54B4FF07E523946009030
:10192000F34804F036F9F3488068F349086000BFD3
:10193000F248007AA84235D0F048057A007A0A28A1
:101940002ED2DFE800F005090D1115191D212529FA
:10195000E548E749886024E0E948E549886020E0F7
:10196000E848E34988601CE0E748E149886018E0FE
:10197000E648DF49886014E0E548DD49886010E00A
:10198000E448DB4988600CE0E348D949886008E016
:10199000E248D749886004E0D448D549886000E02F
:1019A00000BF00BFD548407AB04236D0D348467A0F
:1019B000407A0A282FD2DFE800F0050A0E12161A24
:1019C0001E22262A4FF07C50C949C86024E0D44822
:1019D000C749C86020E0C448C549C8601CE0C84881
:1019E000C349C86018E0C748C149C86014E0C64888
:1019F000BF49C86010E0C548BD49C8600CE0C44894
:101A0000BB49C86008E0C448B949C86004E0B748A9
:101A1000B749C86000E000BF00BFB848407BA042A3
:101A200044D0B648447B0A2C3ED2DFE804F0050AD5
:101A30000F14191F252B3137BA4805900020049048
:101A400033E0B9480590B94804902EE0B8480590B5
:101A5000B648049029E0B7480590B448049024E0C3
:101A60004FF081400590B14804901EE04FF0814056
:101A70000590B148049018E04FF0814005909B48D4
:101A8000049012E04FF081400590AC4804900CE0C7
:101A90004FF081400590AA48049006E04FF0814045
:101AA0000590A848049000E000BF00BF9348007B69
:101AB00050452CD0914890F80CA0007B0A2824D2E5
:101AC000DFE800F005080B0E1114171A1D20642022
:101AD00006901BE03C20069018E01E20069015E0C2
:101AE0001420069012E00F2006900FE00A200690C6
:101AF0000CE00820069009E00620069006E004208D
:101B0000069003E00220069000E000BF00BF7B4883
:101B1000C07A484530D0794890F80B90C07A0B28AD
:101B200028D2DFE800F006090C0F1215181B1E2141
:101B300024006FF0040B1EE06FF0030B1BE06FF04E
:101B4000020B18E06FF0010B15E04FF0FF3B12E0C5
:101B50004FF0000B0FE04FF0010B0CE04FF0020BC9
:101B600009E04FF0030B06E04FF0040B03E04FF0E9
:101B7000050B00E000BF00BFBE2004F039F9FFF7FD
:101B8000EDFD564908600846006805F073FE0746FB
:101B90003946574804F031F8554800685049086004
:101BA0000846006805F02AFE52498968471A3846F7
:101BB00005F00DFBCDE900014E49D1E900733A462D
:101BC000019905F057FBCDE9020105F0C3FA5E4922
:101BD0000860BBF1000F1BD05C4801780078401C06
:101BE0005A4A107006988000814211DD002011468B
:101BF00008704048806840490968884204D13D48DF
:101C0000806858443B4988603A4880683A4908608F
:101C1000049805F063FCCDE902014B4801684C488B
:101C2000006805F08FFF019005F058FC21F000419D
:101C30000746DDE9022305F0E1FA36D24FF0814094
:101C4000059905F077FE0746424908780978491C4E
:101C5000404B197005F026FE8046394605F036FFE8
:101C60002CD200203B490870384908701D48006894
:101C700005F000FE02901A480168029805F057FF2F
:101C800080461C49886805F0F5FD4146039005F043
:101C900051FC074605F0B2FD1649886010480068FF
:101CA00005F0ACFD0F49086008E0002029490870E4
:101CB0000B48006805F0A2FD0A4908602248016847
:101CC0002348006805F03EFF039005F007FC21F073
:101CD000004107464FF080421F4B3FE014000020B8
:101CE0000800002010000020CDCCCC3D6F12833ABC
:101CF000100100202801002024000020B001002055
:101D00000AD7A33D8FC2753D0AD7233D0AD7A33C0E
:101D1000BC74133C4260E53B0AD7A33BA69B443B03
:101D20009A99993E0000A041000070416F12033A59
:101D3000000020410000E04017B7513AA69BC43A8A
:101D40006F12033B0AD7233B0C0000202100002028
:101D50000400002020000020E17A843F05F088FB89
:101D600003D201201749087002E0002015490870CD
:101D7000154801681548006805F0E4FE039005F079
:101D8000ADFB21F0004107464FF06042104B05F0DB
:101D90006FFBBFF4CDAD0F490B48006805F0CAFDDD
:101DA000039005F02BFD804605F064FD07460949C8
:101DB00005F02EFC044908600846006803490860E5
:101DC000B6E50000340000200C00002004000020D4
:101DD0004D62503F00401C4670B50446002503E0AC
:101DE000012003F055FE6D1C4021064801F0BEFDA8
:101DF00008B1A542F4D3A54201D3002070BD012053
:101E0000FCE700000008014070B505460C46284676
:101E100003F0E4FAC4F3074003F0E0FAC4F3072048
:101E200003F0DCFAE0B203F0D9FA70BD70B50446F5
:101E30000D46204603F0D2FA284603F0CFFA70BDD3
:101E400010B51448C06940F001001249C861880407
:101E5000808A40F0010089048882802008800E4832
:101E600000680E49B0FBF1F0401E49060885642069
:101E700088850007808920F0010088810846008855
:101E800020F001000880002088841C2003F058FD09
:101E900010BD000000100240D4000020A086010008
:101EA00010B586B0214C2248806940F4804020491A
:101EB0008861204800684FF4E131B0FBF1F02081E7
:101EC0000020A0812082A082A08940F00800A0818B
:101ED000A08940F00400A081A08940F40050A081B6
:101EE000012240F22551204603F05EFC1048806933
:101EF00040F004000E4988610F48006820F47F60BC
:101F000040F496600C490860252003F019FD00207C
:101F1000029003900490059002A8019001A803F09C
:101F2000C7FF0649086006B010BD00000038014038
:101F300000100240D4000020040801406C00002082
:101F400001461648164AD26942F40032144BDA614F
:101F5000144A1268B2FBF1F2C2F34F02028100226E
:101F6000828102828282828942F008028281828991
:101F700042F004028281828942F4005282811A4630
:101F8000926942F004029A61074A126822F47F4281
:101F900042F49642044B1A6070470000004400402F
:101FA00000100240D40000200008014070B5044633
:101FB0000D460F490F48006803F09CFF00260FE014
:101FC00014F8010B03F060FB02E0322003F060FD27
:101FD0000948008800F040000028F6D0701CC6B206
:101FE000AE42EDDB0348006803F078FF70BD0000EF
:101FF00020A107006C0000200038014000B5024617
:1020000003F036FB107000BDC2B000203F9040903E
:102010003FA83E9000213EA803F078FFFE490860EB
:1020200000BF4FF0FF31FD48006803F091FFFC480E
:102030008078FB49497840EA0120B0F5437F7DD0A4
:1020400048DC40F20122A0EB0201904277D022DC72
:10205000232875D00DDC162873D005DC022871D03A
:10206000142841F06482A0E117286CD02228F8D10E
:1020700089E2B0F5957F67D006DCA0F20110002858
:1020800075D02828EDD1A3E2A0F22B1000286FD044
:102090000128E6D174E340F20112881A914268D017
:1020A0000DDC052975D004DC012973D00229D8D1B3
:1020B000FEE306296FD0B1F5807FD2D1F9E3401F4E
:1020C000052881F03482DFE810F07A0559056F05A4
:1020D0004E05640540F20E52811A904277D025DCFD
:1020E00040F20152A0EB0201904271D013DC40F2A9
:1020F0000342A0EB020190426BD007DCB0F5447FB5
:1021000068D0A0F201400028ABD1D5E3032977D0F5
:102110000729A6D1D1E30729D3D2DFE811F0080AB5
:10212000200644066806080A8C069B0640F2F52045
:102130000A1A814201F072801CDC06E0BEE32DE346
:102140002BE2CDE031E0FCE08BE2B1F5FB7F71D01A
:1021500004DC04296FD0052989D1B0E3A1F2F32171
:10216000002901F03F8001298CD101F049B81EE21D
:1021700005E3A5E340F2FD31501A8A4201F06A817D
:102180000ADC062A01F05880B2F5837F8FD101F076
:1021900020B996E396E396E3012801F05F81A0F26F
:1021A0000510002889D101F068B99E48007890B1E7
:1021B0009DA1A148FEF7C8F89F48FEF72EFAC0B2CD
:1021C00001460F909C48FFF7F1FE01F0B1B97BE3A7
:1021D0007BE37BE37BE34FF07E519848006805F09A
:1021E00075FB0ED296A19448FEF7AEF89248FEF722
:1021F00014FAC0B201460F908F48FFF7D7FEE4E70C
:1022000066E39348007805F04DFB0F908B4801681A
:102210000F9805F05BFB0FD28EA18748FEF794F86C
:102220008548FEF7FAF9C0B201460F908248FFF7E1
:10223000BDFECAE74DE34DE303F024F968B189A17F
:102240007D48FEF781F87C48FEF7E7F9C0B2014609
:102250000F907948FFF7AAFEB7E786A17648FEF708
:1022600073F87548FEF7D9F9C0B201460F9072486D
:10227000FFF79CFE642003F0BBFD0120814908703C
:102280006748007A6649C979654A9279CDE90021A3
:1022900002906348C0786249097940EA01200E90B3
:1022A0005F48407903460F9077A17E480E9AFEF76B
:1022B0004BF800203D900AE059493D980930095CEF
:1022C000794A3D9811543D98401CC0B23D90544805
:1022D0000930FEF7A2F9401E3D998842ECD874E718
:1022E0004F48C0784E49097900EB012080B20F9029
:1022F0000F9818B901206D4948710AE00F986328BA
:1023000003DD63206949487103E00F98C1B2674853
:10231000417166484079024665A10E904648FEF735
:1023200013F84548FEF779F9C0B201460E904248CD
:10233000FFF73CFEC4225D494FF4007001F008FA3B
:1023400043E73748C0783649097900EB012080B26D
:102350000F900F98282803DA2820544908710CE0C0
:10236000584909780F98884204DD564801784F484B
:10237000017102E04D490F9808714C4800790246FE
:1023800051A10E902C48FDF7DFFF2B48FEF745F9D1
:10239000C0B201460E902848FFF708FEC422434908
:1023A0004FF4007001F0D4F90FE700203D90642055
:1023B00003F01EFD49A12048FDF7C6FF1E48FEF7A9
:1023C0002CF9C0B201460F901B48FFF7EFFD00BF8C
:1023D0003D98401CC0B23D90444880680B9005F089
:1023E00049FA0C90424801680C9805F0ABFB0D903F
:1023F00005F074F821F0004100223E4BCDE90E01BA
:1024000005F036F87CD23A48006805F0F7F937490C
:1024100088604FF4167070E0B00000207800002053
:102420004C01002034000020706C617920312C3385
:102430002C30FFFFFF0000000010002004000020EF
:10244000706C617920312C362C30FFFFFF000000CA
:1024500085000020706C617920312C372C30FFFF13
:10246000FF000000706C617920312C382C30FFFFA8
:10247000FF000000706C617920312C352C30FFFF9B
:10248000FF00000084000020253034642D25303208
:10249000642D2530326420253032643A2530326490
:1024A0000000000000030020D8020020B00100203E
:1024B0006D61696E2E6E302E76616C3D2564FFFF76
:1024C000FF000000860000206D61696E2E6E312EC7
:1024D00076616C3D2564FFFFFF0000007473772078
:1024E00062312C30FFFFFF000000000028010020B7
:1024F000080000200000244002E003F079FC13E013
:10250000F5A1FB48FDF720FFF948FEF786F8C0B2B9
:1025100001460F90F648FFF749FD0120F549087084
:102520000020F549088003E03D980C28FFF650AFE5
:1025300000BF3D980C2812DBF0A1ED48FDF704FF29
:10254000EB48FEF76AF8C0B201460F90E848FFF783
:102550002DFD0120E74908700020E7490880EDA122
:10256000E348FDF7F1FEE248FEF757F8C0B2014636
:102570000F90DF48FFF71AFD1022EA494FF4A070D0
:1025800001F0E6F821E6E848C078E8498871C422FD
:102590004FF4007001F0DCF817E6E348C078E34937
:1025A000C871C4224FF4007001F0D2F80DE6DF4884
:1025B0008079012806D1DE48007818B90120DC496D
:1025C000087004E00020DA490870DA490870FCE578
:1025D000D9480168D94805F0B5FA079004F07EFFA4
:1025E000CDE90E01D448006804F078FFCDE90C0174
:1025F000D348006804F072FFCDE90A01D1480068B1
:1026000004F06CFFCDE90801DDE90E01CDE906011A
:10261000DDE90C01CDE90401DDE90A01CDE90201A2
:10262000DDE90801C84BC94ACDE90001C8A1B0489D
:10263000FDF78AFEAE48FDF7F0FFC0B201460F90ED
:10264000AB48FFF7B3FCD2A1A948FDF77DFEA8482F
:10265000FDF7E3FFC0B201460F90A548FFF7A6FCC7
:10266000B3E5B24A2032D2A1A148FDF76DFEA048E1
:10267000FDF7D3FFC0B201460F909D4803F05EF80E
:10268000AA48007F70B1A94A4032D1A19848FDF70D
:102690005BFE9748FDF7C1FFC0B201460F9094481A
:1026A00003F04CF8A148407F70B1A04A6032C8A145
:1026B0008F48FDF749FE8E48FDF7AFFFC0B20146D7
:1026C0000F908B4803F03AF89848807F70B1974A92
:1026D0008032BFA18648FDF737FE8548FDF79DFF94
:1026E000C0B201460F90824803F028F89248016872
:1026F000924805F027FA079004F0F0FECDE90E01AC
:102700008D48006804F0EAFECDE90C018C480068B1
:1027100004F0E4FECDE90A018A48006804F0DEFE18
:10272000CDE90801DDE90E01CDE90601DDE90C0185
:10273000CDE90401DDE90A01CDE90201DDE9080185
:10274000814B824ACDE90001A3496948FDF7FCFDB0
:102750006748FDF762FFC0B201460F90644802F07F
:10276000EDFF9EA16248FDF7EFFD6148FDF755FFC3
:10277000C0B201460F905E4802F0E0FF25E524E577
:102780006A48C07F08B9012000E000206749C87787
:10279000C4224FF4007000F0DBFF16E59AA1544804
:1027A000FDF7D2FD5248FDF738FFC0B201460F9049
:1027B0004F48FFF7FBFB03205E4908705B48007A37
:1027C000024696A10F904A48FDF7BEFD4848FDF726
:1027D00024FFC0B201460F904548FFF7E7FB53487E
:1027E000C07A024694A10F904148FDF7ADFD4048E4
:1027F000FDF713FFC0B201460F903D48FFF7D6FB2F
:102800004A48407A024693A10F903948FDF79CFD53
:102810003748FDF702FFC0B201460F903448FFF77A
:10282000C5FB4248007B024691A10F903048FDF75E
:102830008BFD2F48FDF7F1FEC0B201460F902C48EA
:10284000FFF7B4FB3948807A024690A10F902848E0
:10285000FDF77AFD2648FDF7E0FEC0B201460F9075
:102860002348FFF7A3FB3148407B02468EA10F901F
:102870001F48FDF769FD1E48FDF7CFFEC0B20146B7
:102880000F901B48FFF792FB2848807802468DA1E5
:102890000F901748FDF758FD1548FDF7BEFEC0B272
:1028A00001460F901248FFF781FB2048C07801E0F5
:1028B00027E18FE1024611E1CEE128E248E15DE344
:1028C000A7E122E119E13FE166E324E2E8E1BFE1AB
:1028D00016E265E344E300007431382E7478743DE9
:1028E00022B5F7C1E3B3C9B9A622FFFFFF0000007C
:1028F00000100020AD000020AE0000207431382E02
:102900007478743D22B5F7C1E3CAA7B0DC22FFFF9B
:10291000FF0000007473772062312C31FFFFFF004D
:1029200000000000280100204C010020B001002020
:10293000AC00002084000020980000200000C84265
:10294000940000209000002000030020D802002006
:10295000446174614465616C2E446174614C6F67BD
:102960002E696E73657274282225735E25735E2549
:102970002E3366675E252E3366675E252E3266250A
:10298000255E252E326625252229FFFFFF00000047
:1029900052756E506167652E74382E7478743D22BE
:1029A000B1A3B4E6B3C9B9A62122FFFFFF0000001E
:1029B0002F2A2A2A2A2A2A2A2A2A2A2A2A2A2A2A72
:1029C0002A2A2A2A2A2A2A2A2A2A2A2A2A2F0D0A9F
:1029D000202025730D0A0000987C00082F2A2A2A3F
:1029E0002A2A2A2A2A2A2A2A2A2A2A2A2A2A2A2A47
:1029F0002A2A2A2A2A2A2A2A2A2F0D0A0D0A0D0AE9
:102A00000D0A2000000000007061676520576569AD
:102A1000676874536574FFFFFF00000057656967BE
:102A200068745365742E6362352E76616C3D25643F
:102A3000FFFFFF0000000000576569676874536579
:102A4000742E6362342E76616C3D2564FFFFFF00B7
:102A5000000000005765696768745365742E6362EF
:102A6000332E76616C3D2564FFFFFF0000000000FF
:102A70005765696768745365742E6362322E766198
:102A80006C3D2564FFFFFF0000000000576569678B
:102A900068745365742E6362312E76616C3D2564D3
:102AA000FFFFFF0000000000576569676874536509
:102AB000742E6362302E76616C3D2564FFFFFF004B
:102AC000000000005765696768745365742E6E30A6
:102AD0002E76616C3D2564FFFFFF0000F4A10F908E
:102AE000F948FDF731FCF848FDF797FDC0B2014603
:102AF0000F90F548FFF75AFA22E40420F3490870D2
:102B00001EE40520F14908701AE40820EF49087016
:102B1000EF4AF0A1EC48FDF717FCEB48FDF77DFD0F
:102B2000C0B201460F90E848FFF740FAEFA1E6482F
:102B3000FDF70AFCE448FDF770FDC0B201460F90B6
:102B4000E148FFF733FA2FE40020E04908702BE456
:102B5000EC48C078DE49A0390872C4224FF40070F6
:102B600000F0F6FD20E4E748C078D949A039487262
:102B7000C4224FF4007000F0EBFD15E4E148C0788A
:102B8000D349A0398872C4224FF4007000F0E0FDF0
:102B90000AE4DC48C078CE49A039C872C4224FF498
:102BA000007000F0D5FDEDE4D648C078C849A039E2
:102BB0000873C4224FF4007000F0CAFDE2E4D1486B
:102BC000C078C349A0394873C4224FF4007000F0A4
:102BD000BFFDD7E4CB48C078052804DC0520BC49FC
:102BE000A03988700DE0C748C078782804DD7820C7
:102BF000B749A039887004E0C248C078B449A03908
:102C00008870C422B249A0394FF4007000F0A0FDD2
:102C1000B8E4BC48C078052804DC0520AC49A039DC
:102C2000C8700DE0B748C078C82804DDC820A8499E
:102C3000A039C87004E0B348C078A549A039C8706D
:102C4000C422A349A0394FF4007000F081FD99E43B
:102C500002209E49087095E49D48A038006901460D
:102C60000D90A948006804F06DFF0F90A548C0784A
:102C7000A449097900EB01200C9004F0FBFDA34965
:102C80000D9004F0C5FC0E900F9904F05BFF904985
:102C9000A0390861C4224FF4007000F059FD71E4BE
:102CA0009B48006804F0AAFD9A498968401A0C9074
:102CB00004F0E0FD0E909348C0789249097900EB4A
:102CC00001209049497900EB01408E49897900EB58
:102CD00001600B9004F0CEFD8F490C9004F098FC3D
:102CE0000D900E9904F094FC0F9004F0F7FB894AC4
:102CF00003C2102287494FF4A07000F029FD41E47F
:102D00008348006804F07AFD824988603AE4022032
:102D10006E49087036E400203D900BE079493D98FB
:102D2000C01C0A5C6A4880383D9942543D98401C5A
:102D3000C0B23D907348C01CFDF76FFC401E3D992A
:102D40008842EBD80022624880383D994254C42220
:102D5000A0F120014FF4007000F0FAFCE8E300203D
:102D60003D900BE067493D98C01C0A5C58486038AC
:102D70003D9942543D98401CC0B23D906148C01CF2
:102D8000FDF74BFC401E3D998842EBD8002250488D
:102D900060383D994254C422A0F140014FF40070C4
:102DA00000F0D6FCC4E300203D900BE055493D986F
:102DB000C01C0A5C464840383D9942543D98401C2E
:102DC000C0B23D904F48C01CFDF727FC401E3D9906
:102DD0008842EBD800223E4840383D994254C422F4
:102DE000A0F160014FF4007000F0B2FCA0E30020FD
:102DF0003D900BE043493D98C01C0A5C34482038A4
:102E00003D9942543D98401CC0B23D903D48C01C85
:102E1000FDF703FC401E3D998842EBD800222C4868
:102E200020383D994254C422A0F180014FF4007033
:102E300000F08EFC7CE33348C07808B1012000E04C
:102E400000202349A0390877C4224FF4007000F015
:102E50007FFC6DE32B48C0782A49097900EB0120FB
:102E60002849497900EB01402649897900EB016046
:102E7000082862D2DFE800F0040A101652575C629C
:102E80004FF496601249A03988615CE04FF41660F7
:102E90000F49A039886156E04FF496500C49A0398B
:102EA000886150E04FF416500949A03988614AE022
:102EB0005765696768745365742E6E312E76616C40
:102EC0003D2564FFFFFF000000100020840000206B
:102ED000500200205379735365742E7431342E746C
:102EE00078743D22257322FFFFFF0000537973534E
:102EF00065742E74302E7478743D2222FFFFFF001B
:102F0000000000004C01002068000020000020416B
:102F1000080000202801002000401C464FF4964085
:102F2000F84988610FE04FF41640F64988610AE0DD
:102F30004FF46140F349886105E000BF4FF4E13090
:102F4000F049886100BF00BFC422EE494FF4007011
:102F500000F0FEFBEB4880690F90FEF7F1FFE7E21F
:102F6000E948C07808B1012000E00020E549487731
:102F7000C4224FF4007000F0EBFBD9E2E248C078C5
:102F800008B1012000E00020DE498877C4224FF418
:102F9000007000F0DDFBCBE20220DC490870C7E2E4
:102FA00000203D900AE0D8493D98C01C095CD84AF1
:102FB0003D9811543D98401CC0B23D90D248C01C71
:102FC000FDF72BFB401E3D998842ECD800203D9038
:102FD0003C9000BF3D98411CC9B23D91CC490A5C70
:102FE0003C98411CC9B23C9134A90A54C8493D9847
:102FF000085C5E28EED13D98401CC0B23D90002098
:103000003C9000BF3D98411CC9B23D91C0490A5C4B
:103010003C98411CC9B23C912CA90A54BC493D982A
:10302000085C5E28EED13D98401CC0B23D90002067
:103030003C9000BF3D98411CC9B23D91B4490A5C27
:103040003C98411CC9B23C9127A90A54B0493D980B
:10305000085C5E28EED13D98401CC0B23D90002037
:103060003C9000BF3D98411CC9B23D91A8490A5C03
:103070003C98411CC9B23C9122A90A54A4493D98EC
:10308000085C5E28EED13D98401CC0B23D90002007
:103090003C9000BF3D98411CC9B23D919C490A5CDF
:1030A0003C99481CC0B23C901DA8425498493D9898
:1030B000085C5E28EED13D98401CC0B23D900020D7
:1030C0003C9000BF3D98411CC9B23D9190490A5CBB
:1030D0003C98411CC9B23C9118A90A548C48FDF790
:1030E0009CFA3D998842EDD8864A2032AFF2407171
:1030F0008848FDF729F98748FDF78FFAC0B20146E5
:103100000F90844802F01AFBC82002F071FE7D483F
:10311000007F90B17B4A4032AFF24C717D48FDF7A1
:1031200013F97C48FDF779FAC0B201460F9079484F
:1031300002F004FBC82002F05BFE7248407F90B1B1
:10314000704A6032AFF278717248FDF7FDF871484D
:10315000FDF763FAC0B201460F906E4802F0EEFA36
:10316000C82002F045FE6748807F90B1654A8032F2
:10317000AFF2A4716748FDF7E7F86648FDF74DFA2E
:10318000C0B201460F90634802F0D8FAC82002F09E
:103190002FFE18A81DA922AA27ABCDE90032CDE940
:1031A00002102CAB34AA5C495A48FDF7CDF85948B7
:1031B000FDF733FAC0B201460F90564802F0BEFA4E
:1031C000C82002F015FEAFF2EC715248FDF7BCF8D2
:1031D0005048FDF722FAC0B201460F904D4802F068
:1031E000ADFAA5E14DA14B48FDF7AEF84948FDF712
:1031F00014FAC0B201460F904648FEF7D7FE97E199
:103200004AA14448FDF7A0F84248FDF706FAC0B2CB
:1032100001460F903F48FEF7C9FE89E146A13D48AF
:10322000FDF792F83B48FDF7F8F9C0B201460F9060
:103230003848FEF7BBFE7BE100203C9003203D9028
:1032400000BF3D98411CC9B23D912F490A5C3C9892
:10325000411CC9B23C9114A90A542B493D98085C01
:103260005E28EED100203C903D98401CC0B23D90BD
:1032700000BF3D98411CC9B23D9123490A5C3C986E
:10328000411CC9B23C9110A90A541F48FDF7C5F969
:10329000401E3D998842ECD81A49A03114A8FDF788
:1032A000DBF970BB1749B03110A8FDF7D5F940BB69
:1032B00014AA25A11748FDF747F81648FDF7ADF900
:1032C000C0B201460F901348FEF770FE25A11148C9
:1032D000FDF73AF80F48FDF7A0F9C0B201460F908C
:1032E0000C48FEF763FE25A10A48FDF72DF80948B2
:1032F000FDF793F9C0B201460F900648FEF756FE5F
:1033000048E058E0B00100204C010020840000207B
:103310007402002000100020047D000870616765C1
:1033200020537973536574FFFFFF00007061676578
:1033300020564CFFFFFF0000706167652041626FFF
:103340007574FFFFFF000000557365724C6F67498D
:103350006E2E7431342E7478743D2573FFFFFF0098
:1033600000000000557365724C6F67496E2E743013
:103370002E7478743D2222FFFFFF000055736572A2
:103380004C6F67496E2E74332E7478743D2222FF81
:10339000FFFF00006AA16F48FCF7D6FF6D48FDF7FC
:1033A0003CF9C0B201460F906A48FEF7FFFD0920C4
:1033B000694908700CE069A16648FCF7C5FF6548DB
:1033C000FDF72BF9C0B201460F906248FEF7EEFD03
:1033D000AEE000203C9003203D9000BF3D98411C92
:1033E000C9B23D9161490A5C3C98411CC9B23C910B
:1033F00014A90A545D493D98085C5E28EED100206E
:103400003C903D98401CC0B23D9000BF3D98411C8F
:10341000C9B23D9155490A5C3C99481CC0B23C90E8
:1034200010A842545148FDF7F8F8401E3D998842D3
:10343000ECD814A94E48FDF7CCF810A94C48103030
:10344000FDF7C7F8C4224A49A0394FF4007000F0D4
:103450007FF900BF00204049087069E0444A45A157
:103460003C48FCF771FF3B48FDF7D7F8C0B2014676
:103470000F903848FEF79AFD5AE000203C90032058
:103480003D9000BF3D98411CC9B23D9137490A5C4F
:103490003C98411CC9B23C9114A90A5433493D9847
:1034A000085C5E28EED100203C903D98401CC0B2E4
:1034B0003D9000BF3D98411CC9B23D912B490A5C2B
:1034C0003C99481CC0B23C9010A842542748FDF7D4
:1034D000A4F8401E3D998842ECD8254914A8FDF770
:1034E000BBF8B0B92249103110A8FDF7B5F880B982
:1034F00026A11848FCF728FF1648FDF78EF8C0B241
:1035000001460F901348FEF751FD00201249087044
:103510000CE012A10F48FCF717FF0E48FDF77DF8ED
:10352000C0B201460F900B48FEF740FD00BF00BF40
:1035300000BF1A48006802F0FFFCFEF772BD0000F1
:103540007061676520557365724C6F67496EFFFF48
:10355000FF0000000010002084000020706C6179E2
:1035600020312C312C30FFFFFF0000004C010020E7
:10357000500200204C6F67496E2E7431342E7478DF
:10358000743D22257322FFFFFF0000007061676514
:10359000206D61696EFFFFFF00000000B000002099
:1035A00070B5C4223D494FF4007000F0A3F8C42266
:1035B0003A494FF4007000F09DF8102238494FF45A
:1035C000A07000F097F83648364A374BD0E90041F2
:1035D000204603F013FE03D232483349304A03C277
:1035E0002E48008845F2AA51884206D12B48B0F8EF
:1035F000C0004AF6552188424FD045F2AA502749CB
:1036000008803C2088700520C8706920087105205A
:10361000487100208871C871052008720220487224
:10362000052088720620C87208200873002048739D
:10363000086148614FF41650886100200877487788
:103640008877C87719A115482030FCF77DFE1AA1AC
:1036500012484030FCF778FE16A110486030FCF7A5
:1036600073FE14A10D488030FCF76EFE19A10B48C3
:10367000A030FCF769FE19A10848B030FCF764FEE1
:103680004AF655200549A1F8C00081071548044AAB
:10369000C2E9001014481146886070BDB0010020D6
:1036A0002801002048AFBC9AF2D77A3EB2E2CAD4D1
:1036B000BDE1B9FB00000000C9BDB6ABD4C6CCC6A5
:1036C000D6C7C4DCBFC6BCBCD3D0CFDEB9ABCBBE83
:1036D00000000000CAB5D1E9CAD20000313233344B
:1036E000353600008171153FD65F0B0010B500F034
:1036F000ABFA10BD70B504460D46164600F048FB07
:10370000A02000F011FB00F07DFB201200F00CFB6C
:1037100000F078FBE0B200F007FB00F073FB00F074
:1037200037FBA12000F000FB00F06CFB08E00EB1BD
:10373000012100E00021084600F0C4FA05F8010B61
:10374000301EA6F10101CEB2F1D100F03FFB70BDF9
:1037500070B504460D46164600F01AFBA02000F096
:10376000E3FA00F04FFB201200F0DEFA00F04AFB13
:10377000E0B200F0D9FA00F045FB05E015F8010BC6
:1037800000F0D2FA00F03EFB301EA6F10101CEB2ED
:10379000F4D100F01BFB70BD08B50121082001F039
:1037A000CBFD4FF47040ADF8000048208DF80300C9
:1037B00003208DF802006946014800F003F808BDB7
:1037C000000C01402DE9F0410246002500260020B2
:1037D00000230024002791F803C00CF00F0591F896
:1037E00003C00CF0100CBCF1000F03D091F802C024
:1037F0004CEA050591F800C0BCF1000F31D0146807
:1038000000202BE04FF0010C0CFA00F3B1F800C0DF
:103810000CEA03069E4220D183004FF00F0C0CFAF5
:1038200003F7BC4305FA03FC4CEA040491F803C017
:10383000BCF1280F06D14FF0010C0CFA00FCC2F8C5
:1038400014C00AE091F803C0BCF1480F05D14FF055
:10385000010C0CFA00FCC2F810C0401C0828D1D39F
:103860001460B1F800C0BCF1FF0F34DD54680020D3
:103870002EE000F1080C4FF0010808FA0CF3B1F843
:1038800000C00CEA03069E4221D183004FF00F0CCA
:103890000CFA03F7BC4305FA03FC4CEA040491F864
:1038A00003C0BCF1280F05D100F1080C08FA0CF890
:1038B000C2F8148091F803C0BCF1480F07D100F1A1
:1038C000080C4FF0010808FA0CF8C2F81080401CF0
:1038D0000828CED35460BDE8F0810000F0B50A4658
:1038E000002300240021002500F00046B6F1004F1F
:1038F00002D11D4EF16901E01B4E7168C0F3034512
:1039000083B200F44016B6F5401F08D121F0706173
:10391000154E766826F07066134F7E6012E000F454
:103920008016B6F5801F06D1032606FA05F4A143DA
:1039300041F0706106E0460D360103FA06F6B14328
:1039400041F0706122B1460D360103FA06F63143AB
:1039500000F00046B6F1004F02D1034EF16101E0E4
:10396000014E7160F0BD00000000014002460020E1
:1039700093680B400BB1012000E0002070474161CB
:10398000704701617047000010B50021024802F045
:10399000EBFA01F0B5FC10BD887C00082DE9F04F72
:1039A0008DB04FF00009002500200B9083460A904F
:1039B00009900890794807907949087903F072FFD7
:1039C0000C907848784908607848794908604FF049
:1039D0007E50784908600020774908607749088060
:1039E0004FF4FA7002F004FA0120FDF707FE4FF4DD
:1039F000FA7002F0FDF902F04FFA06907048008864
:103A00004FF47A7148436F4909884FF47A725143F1
:103A100000EB1146ABE06C48D0F80080AA46414666
:103A20000C9804F08FF805466849284604F04EF8D3
:103A30000ED26748006881465F490860654948467C
:103A400003F078FF049003F0F5FE5C49088073E012
:103A500029465548006803F06DFF0B9029465448ED
:103A6000006803F067FF5946049003F063FD834646
:103A70005949584603F02AFF01D2DFF85CB14FF0F4
:103A80007E51584604F022F801D24FF07E5B514639
:103A9000284604F057F8019046480168019803F061
:103AA00049FF4E49029003F045FF4D4904900A98A2
:103AB00003F040FF0390049903F03CFD0A904FF09F
:103AC0007E50079904F03EF8594602900B9803F097
:103AD00031FD00900A9903F02DFD0190029903F049
:103AE00029FF04900799099803F024FF0390049993
:103AF00003F020FD0990DDE9081003F01BFD81466D
:103B00000021484603F0E2FE01D24FF000093048A0
:103B10000168484603F0DAFF02D22D48D0F8009041
:103B20002548C0F800902B49484603F003FF049055
:103B300003F080FE2149088002F0AEF90446A01986
:103B4000401E0699401AB0FBF6F7B7F5967F03D2F0
:103B5000C7F59670059002E006941E200590059822
:103B600002F046F9DDE9050100FB061006901D484C
:103B7000007801283FF44FAF00200F4908600F493B
:103B800008804FF4FA7002F033F90020FDF736FD9B
:103B90000020144908700DB0BDE8F08FCDCC4C3F2B
:103BA000B00100208FC2753D50000020240B9839D1
:103BB0005400002058000020600000203800002041
:103BC000747D0008767D0008680000200000A04198
:103BD0006400002000007A44000080BFFA7EAA3E04
:103BE00083C02A3F5C00002010B50021014802F08C
:103BF000BBF910BD547C000870B50546FFF7CEFE3A
:103C000002F0D4F9044602F0DDF970BD10B54FF4AE
:103C100080710C48FFF7B3FE4FF400710948FFF7BD
:103C2000AEFE012001F034FF4FF480710548FFF72C
:103C3000A8FE012001F02CFF4FF480710148FFF72E
:103C40009EFE10BD000C014008B50121082001F0C6
:103C500073FB4FF44070ADF8000014208DF80300A2
:103C600003208DF8020069460648FFF7ABFD4FF4CC
:103C700000710448FFF785FE4FF480710148FFF79B
:103C800080FE08BD000C014010B54FF480710C4857
:103C9000FFF775FE4FF400710948FFF772FE01202F
:103CA00001F0F6FE4FF480710548FFF76AFE01202F
:103CB00001F0EEFE4FF480710148FFF760FE10BD89
:103CC000000C014070B5054600244FF40071154802
:103CD000FFF757FE00261BE04FF480711148FFF7F5
:103CE0004EFE012001F0D4FE6006040E4FF48071F8
:103CF0000C48FFF746FE012001F0CAFE4FF40071A8
:103D00000848FFF733FE08B144F00104701CC6B246
:103D1000082EE1DB15B9FFF7B7FF01E0FFF776FFEB
:103D2000204670BD000C014070B504464FF4807110
:103D30001648FFF724FE012001F0AAFE002521E02D
:103D400004F0800028B14FF400711048FFF719FE0D
:103D500004E04FF400710D48FFF711FE012001F05F
:103D600097FE4FF480710948FFF70BFE012001F028
:103D70008FFE4FF480710548FFF701FE6006040EC8
:103D8000681CC5B2082DDBDB70BD0000000C0140D3
:103D900010B54FF400710C48FFF7F3FD4FF480713C
:103DA0000948FFF7EEFD012001F072FE4FF40071AB
:103DB0000548FFF7E4FD012001F06AFE4FF4807131
:103DC0000148FFF7DCFD10BD000C014010B54FF4B9
:103DD00080710B48FFF7D3FD4FF400710848FFF7DF
:103DE000CEFD012001F054FE4FF480710448FFF72E
:103DF000C8FD4FF400710248FFF7C3FD10BD00007D
:103E0000000C014010B500244FF400711548FFF775
:103E1000B8FD012001F03CFE4FF480711148FFF71E
:103E2000B0FD012001F034FE0AE0012001F030FE77
:103E3000601CC4B2FA2C03DDFFF7C8FF012010BDDF
:103E40004FF400710748FFF791FD0028EDD14FF4C2
:103E500080710448FFF793FD012001F019FE002056
:103E6000EDE70000000C014010B54FF480510D4803
:103E7000FFF77CFD04464FF400510A48FFF776FD3A
:103E800044EA40044FF480410648FFF76FFD44EADE
:103E900080044FF400410348FFF768FD44EAC00086
:103EA000C0B210BD000C014008B51A481A4B4FF0C3
:103EB0007E5200210090194801F064FE00BFFA20F4
:103EC00001F096FF00F064F80446E510C4F38006A4
:103ED000284603F0E7FC80464FF07A5103F02AFDB4
:103EE000074656B1E843401C03F0C4FC80464FF03F
:103EF0007A5103F01FFD80F000473946074801F072
:103F00004FFE074A1169054A106803F013FB054983
:103F10000860D4E79A99993E0AD7233C38010020DB
:103F2000B00100206800002008B510211648FFF7F6
:103F300028FD2020ADF8000010208DF8030003209C
:103F40008DF8020069461048FFF73CFC1020ADF8E0
:103F500000008DF8030003208DF8020069460A482E
:103F6000FFF730FC0820ADF8000004208DF80300B6
:103F700003208DF8020069460348FFF723FC002167
:103F8000024801F0F1FF08BD000C0140647C00080C
:103F900070B50025002410211248FFF7F0FC0F2413
:103FA00018E020210F48FFF7EAFC012001F070FD26
:103FB00008210C48FFF7DAFC18B10120A040284383
:103FC00085B220210748FFF7DCFC012001F060FDED
:103FD000601E44B2002CE4DA10210248FFF7D1FC45
:103FE000284670BD000C01408CB000200B9064206E
:103FF0000A90F948C07F0990FFF7D2FA4FF47A701F
:1040000001F0F6FEF548006803F0F8FBF44988601B
:10401000F14880690790FDF793FF00200890F14870
:10402000006803F05BFACDE9060101460798CDE987
:104030000010ED480278EDA1F548FCF785F9F44849
:10404000FCF7EBFAC0B201460790F148FDF7AEFF6E
:104050004FF4967001F0CCFEE248006803F03EFA9F
:10406000CDE90601CDE90001DF480278E9A1E84881
:10407000FCF76AF9E648FCF7D0FAC0B201460790AF
:10408000E348FDF793FF00BFEC480078002873D1A8
:10409000D148C0790246EAA10790DD48FCF754F9FF
:1040A000DB48FCF7BAFAC0B201460790D848FDF7E2
:1040B0007DFFC94800790246E6A10790D448FCF785
:1040C00043F9D348FCF7A9FAC0B201460790D0489B
:1040D000FDF76CFFC04880790246E3A10790CC4809
:1040E000FCF732F9CA48FCF798FAC0B201460790CB
:1040F000C748FDF75BFFB84840790246DFA107904B
:10410000C348FCF721F9C248FCF787FAC0B2014660
:104110000790BF48FDF74AFF4FF08041B148006863
:1041200003F076FA0390DA480168039803F002FA84
:104130000490AC480168049803F06AFA059003F013
:104140005DFB069003F096FB0790A6480168079870
:1041500003F0F0FB0890A448007803F0A3FB07905D
:10416000089903F0B3FC0DD8089803F0B7F902469C
:104170000B46CDE9060100E0D1E0C6A1A448FCF75A
:10418000E3F803E0C9A1A248FCF7DEF8A048FCF779
:1041900044FAC0B2014607909D48FDF707FF8E4ADA
:1041A000A032C9A19A48FCF7CFF89948FCF735FA34
:1041B000C0B2014607909648FDF7F8FEC84800686F
:1041C00003F08CF902460B46CDE90601C5A19048E3
:1041D000FCF7BAF88E48FCF720FAC0B20146079007
:1041E0008B48FDF7E3FEC6A18948FCF7ADF8884887
:1041F000FCF713FAC0B2014607908548FDF7D6FEDA
:1042000088E0C348007801281DD1C2480188008891
:10421000401CC04A1080052918DD0020BC490870E8
:1042200011460880BCA17A48FCF78EF87848FCF764
:10423000F4F9C0B2014607907548FDF7B7FE642057
:1042400001F0D6FD02E00020B24908804FF0804125
:104250006448006803F0DCF903908D480168039816
:1042600003F068F904905F480168049803F0D0F9FE
:10427000059003F0C3FA069003F0FCFA0790594842
:104280000168079803F056FB08905748007803F040
:1042900009FB0790089903F019FC0BD8089803F064
:1042A0001DF902460B46CDE906017AA15848FCF7F4
:1042B0004BF803E07DA15648FCF746F85448FCF75C
:1042C000ACF9C0B2014607905148FDF76FFE0B985C
:1042D000411CC9B20B91032816DD00200B908048C9
:1042E000006803F0FBF802460B46CDE906017DA10C
:1042F0004748FCF729F84648FCF78FF9C0B2014659
:1043000007904348FDF752FE4FF4967186480068C7
:1043100001F01EFE4948007800283FF472AF47487C
:104320000078012857D10020804908808049088002
:104330004FF080412B48006803F06AF9029054481E
:104340000168029803F0F6F8039026480168039884
:1043500003F05EF9049003F051FA059003F08AFA35
:10436000069020480168069803F0E4FA0890714925
:10437000089808601848C07920B1012807D00228A1
:104380000FD109E04FF07E506B4908600AE04FF012
:104390007D506949086005E04FF07C50664908602F
:1043A00000E000BF00BF0C48C07F08B163A000E080
:1043B00064A0024665A106901548FBF7C5FF1448A6
:1043C000FCF72BF9C0B2014606901148FDF7EEFD4F
:1043D000014AA032C6E0FDE3B00100200800002041
:1043E0002801002088000020850000206D61696E92
:1043F0002E74362E7478743D224D61783D256467A5
:1044000020443D25312E33666722FFFFFF00000068
:104410000012002052756E506167652E74362E743E
:1044200078743D224D61783D25646720443D2531F7
:104430002E33666722FFFFFF00000000840000208B
:104440006D61696E2E6362312E76616C3D2564FF6D
:10445000FFFF00006D61696E2E6E312E76616C3D3E
:104460002564FFFFFF0000006D61696E2E636230FE
:104470002E76616C3D2564FFFFFF00006D61696E63
:104480002E6E302E76616C3D2564FFFFFF0000002C
:10449000040000206D61696E2E74302E7478743DB6
:1044A0002225332E336622FFFFFF00006D61696E07
:1044B0002E74302E7478743D222D2D2D2E2D2D2D01
:1044C00022FFFFFF000000006D61696E2E74352E23
:1044D0007478743D22257322FFFFFF000000000066
:1044E000680000206D61696E2E7431322E7478740C
:1044F0003D2225332E306622FFFFFF000000000022
:1045000070616765206D61696EFFFFFF000000004C
:10451000AD000020AE0000207431382E7478743D58
:10452000222022FFFFFF0000B0000020A200002098
:10453000A00000209000002064000020BAACB9CC9C
:10454000C1BF0000BAACCBAEC1BF000052756E5007
:104550006167652E74372E7478743D22257322FFAF
:10456000FFFF0000F8A1FE48FBF7EEFEFC48FCF759
:1045700054F8C0B201460690F948FDF717FDF94A14
:10458000F9A1F748FBF7E0FEF548FCF746F8C0B2A2
:1045900001460690F248FDF709FDFA48C079024647
:1045A000F9A10690EE48FBF7CFFEED48FCF735F891
:1045B000C0B201460690EA48FDF7F8FCF1480079E0
:1045C0000246F7A10690E648FBF7BEFEE448FCF77A
:1045D00024F8C0B201460690E148FDF7E7FCE9483F
:1045E00080790246F4A10690DD48FBF7ADFEDC4879
:1045F000FCF713F8C0B201460690D948FDF7D6FC87
:10460000E04840790246F2A10690D548FBF79CFEAF
:10461000D348FCF702F8C0B201460690D048FDF737
:10462000C5FC00F02FFFC0B1EFA1CD48FBF78CFE19
:10463000CB48FBF7F2FFC0B201460690C848FDF731
:10464000B5FC00BF4FF4967001F0D2FB00F01AFFEA
:1046500018B1E94800780128F4D0012000F058FE94
:104660004FF44871E548006801F072FCE4A1BC48D1
:10467000FBF76AFEBA48FBF7D0FFC0B201460690CE
:10468000B748FDF793FCE2A1B548FBF75DFEB448DF
:10469000FBF7C3FFC0B201460690B148FDF786FCA8
:1046A000D7A1AF48FBF750FEAD48FBF7B6FFC0B24D
:1046B00001460690AA48FDF779FCDAA1A848FBF765
:1046C00043FEA748FBF7A9FFC0B201460690A448E5
:1046D000FDF76CFCD7A1A248FBF736FEA048FBF71C
:1046E0009CFFC0B2014606909D48FDF75FFCD5498E
:1046F00008980860D4490860D44800884FF47A715B
:104700004843D34909884FF47A72514300EB114072
:10471000079001F0C1FBCF49086000BF00F0B2FE76
:10472000F0B1B1A18E48FBF70FFE8D48FBF775FF86
:10473000C0B2014606908A48FDF738FC002000F020
:10474000E7FD00BF4FF4967001F052FB00F09AFEB7
:1047500018B1A94800780128F4D0012000F0D8FD54
:1047600001F09AFB079900EB5100BA490968411A18
:104770000798B1FBF0F0B849086008460068B0F54A
:10478000967F0BD208460068C0F59670069001F03F
:104790002FFB01F081FBAF49086006E01E2001F00D
:1047A00027FB01F079FBAB490860A7480068AB49DB
:1047B00008607448807920B1012812D0022824D1E1
:1047C00010E0A74801880088401CA54A10806D4869
:1047D000807800EB4000814202DD0120A149087091
:1047E00014E013E0A04801880088401C9E4A108015
:1047F00064484079C0EB0010800000EB400081422B
:1048000002DD01209749087000E000BF00BF954815
:10481000007800285BD095A15148FBF795FD5048E2
:10482000FBF7FBFEC0B2014606904D48FDF7BEFB0C
:10483000002000F06DFD93A14948FBF785FD484835
:10484000FBF7EBFEC0B2014606904548FDF7AEFB14
:1048500095A14348FBF778FD4148FBF7DEFEC0B267
:10486000014606903E48FDF7A1FB93A13C48FBF7AB
:104870006BFD3B48FBF7D1FEC0B2014606903848BD
:10488000FDF794FB90A13648FBF75EFD3448FBF73B
:10489000C4FEC0B2014606903148FDF787FB8EA1E9
:1048A0002F48FBF751FD2E48FBF7B7FEC0B201467B
:1048B00006902B48FDF77AFB00BF4FF0FF314F48C1
:1048C000006801F045FB4C4800780128F5D04FF016
:1048D00080418548006802F09BFE02908348016891
:1048E000029802F027FE03907F480168039802F0C7
:1048F0008FFE049002F082FF059002F0BBFF06904D
:1049000079480168069803F015F808900021774867
:10491000006803F0DBF815D84A480899006803F0EE
:1049200011F9069070480168069803F0CFF802D29A
:104930004549089808601348C0784FF47A7190FB95
:10494000F1F0D5E014E1000052756E506167652EFC
:1049500074352E7478743D22257322FFFFFF00000A
:1049600000120020D802002052756E506167652E3B
:104970007431342E7478743D22257322FFFFFF00BA
:1049800000000000B001002052756E506167652E76
:104990006362302E76616C3D2564FFFFFF000000EE
:1049A00052756E506167652E6E322E76616C3D25B4
:1049B00064FFFFFF0000000052756E506167652EB6
:1049C0006362312E76616C3D2564FFFFFF000000BD
:1049D00052756E506167652E6E332E76616C3D2583
:1049E00064FFFFFF00000000706C617920312C38FB
:1049F0002C30FFFFFF00000084000020B0000020EA
:104A0000636C652073302E69642C30FFFFFF00005B
:104A1000706167652052756E50616765FFFFFF002A
:104A2000000000007661302E76616C3D30FFFFFFA4
:104A300000000000746D302E656E3D31FFFFFF00F9
:104A4000000000009C000020A8000020747D0008E9
:104A5000767D0008B4000020B800002094000020FB
:104A6000A0000020AC000020A200002052756E5073
:104A70006167652E746D302E656E3D30FFFFFF005F
:104A80000000000052756E506167652E74382E74F8
:104A900078743D22B2E2CAD4D2D1CDEAB3C9212280
:104AA000FFFFFF0000000000706C617920312C34A2
:104AB0002C30FFFFFF0000007473772062302C3130
:104AC000FFFFFF00000000007473772062332C3179
:104AD000FFFFFF00000000007473772062312C316B
:104AE000FFFFFF00000000008800002004000020FD
:104AF000049002F0BFFE0690F4480899006803F0A5
:104B000021F80590069902F0E1FF07D20020F04954
:104B10000880EE4908980860EE4908600021EE48D8
:104B2000006802F037FE23D0EA480168EA480068CE
:104B300003F008F80190E8480168019802F068FD68
:104B4000E649029002F0F6FE0390E54801680398FA
:104B500002F05EFD049002F06DFE059002F0A2FEF0
:104B60000690DF480168069802F0E4FEDD4908601F
:104B7000D848006802F0B2FC02460B46CDE90401B9
:104B8000D9A1E048FBF7E0FBDE48FBF746FDC0B2E9
:104B900001460690DB48FDF709FADB48006802F0A1
:104BA0009DFC02460B46CDE90401D8A1D548FBF790
:104BB000CBFBD448FBF731FDC0B201460690D1488B
:104BC000FDF7F4F9D848C17F099881421CD0D64836
:104BD000C07F00E0BEE00990D348C07F10B1AFF2C3
:104BE000A46001E0AFF2A4600246AFF2A0610690BB
:104BF000C448FBF7A9FBC348FBF70FFDC0B2014651
:104C00000690C048FDF7D2F9C748C07F28B1B54823
:104C10000168B24802F096FF01E0B24800680390D4
:104C200002F05CFC02460B46CDE90401BFA1B54889
:104C3000FBF78AFBB348FBF7F0FCC0B201460690D5
:104C4000B048FDF7B3F9A748006802F0F3FDC0B221
:104C50000246BEA10690AB48FBF776FBA948FBF7DE
:104C6000DCFCC0B201460690A648FDF79FF9BD489E
:104C700001780078401CBB4A1070032953DB0020E8
:104C800011460870B8499748006802F01FFE01D825
:104C9000C8200A90B4499348006802F017FF07D271
:104CA000B2499048006802F011FE01D264200A90D7
:104CB000AE498C48006802F009FF01D246200A90F4
:104CC000AB4909880A98884211D0A9490A980880F6
:104CD00008460288A7A18B48FBF736FB8948FBF7FB
:104CE0009CFCC0B2014606908648FDF75FF97B49FF
:104CF0007C48006802F08CFCA249049002F01AFE85
:104D0000059002F097FDC0B202469FA106907D4833
:104D1000FBF71AFB7B48FBF780FCC0B2014606900C
:104D20007848FDF743F99D48007801283FF4F6AC38
:104D3000AFF2C0217348FBF707FB7248FBF76DFC2D
:104D4000C0B2014606906F48FDF730F9002000F030
:104D5000DFFA00BF9148007803287DD14FF49671A7
:104D60008F48006801F0F4F8002875DD322001F06A
:104D70003FF86D48007A02468AA107906148FBF728
:104D8000E3FA6048FBF749FCC0B2014607905D4872
:104D9000FDF70CF96448C07A024689A1079059488A
:104DA000FBF7D2FA5748FBF738FCC0B20146079030
:104DB0005448FDF7FBF85C48407A024687A107900B
:104DC0005048FBF7C1FA4F48FBF727FCC0B2014639
:104DD00007904C48FDF7EAF85348007B024686A14D
:104DE00007904848FBF7B0FA4648FBF716FCC0B2FC
:104DF000014607904348FDF7D9F84B48807A0246B0
:104E000084A107903F48FBF79FFA3E48FBF705FC5B
:104E1000C0B2014607903B48FDF7C8F84248407BC6
:104E2000024683A107903748FBF78EFA3548FBF717
:104E3000F4FBC0B2014607903248FDF7B7F83A4894
:104E40008078024681A107902E48FBF77DFA2D4815
:104E5000FBF7E3FBC0B200E015E0014607902948EC
:104E6000FDF7A4F83048C07802467EA10790254897
:104E7000FBF76AFA2348FBF7D0FBC0B20146079064
:104E80002048FDF793F84548007804281DD17B4859
:104E9000006802F023FB02460B46CDE9060178A12B
:104EA0001848FBF751FA1748FBF7B7FBC0B20146A9
:104EB00007901448FDF77AF81348006802F00EFBDB
:104EC00002460B46CDE90601EAE0FCE09C0000202A
:104ED000A0000020A8000020900000200000C84290
:104EE0008C0000209800002052756E506167652E7E
:104EF00074302E7478743D2225332E336622FFFFE2
:104F0000FF000000001200206800002052756E5063
:104F10006167652E7431322E7478743D2225332EEC
:104F2000306622FFFFFF0000B001002052756E5076
:104F30006167652E7431372E7478743D2225322EC8
:104F40003266252522FFFFFF0000000052756E50DB
:104F50006167652E6A302E76616C3D2564FFFFFF28
:104F600000000000A4000020000018420000984249
:104F7000A600002073302E6469733D2564FFFFFF97
:104F80000000000000007F436164642073302E69DC
:104F9000642C302C2564FFFFFF00000084000020FB
:104FA000B00000205765696768745365742E6362AA
:104FB000352E76616C3D2564FFFFFF000000000088
:104FC0005765696768745365742E6362342E766121
:104FD0006C3D2564FFFFFF00000000005765696716
:104FE00068745365742E6362332E76616C3D25645C
:104FF000FFFFFF0000000000576569676874536594
:10500000742E6362322E76616C3D2564FFFFFF00D3
:10501000000000005765696768745365742E636209
:10502000312E76616C3D2564FFFFFF00000000001B
:105030005765696768745365742E6362302E7661B4
:105040006C3D2564FFFFFF000000000057656967A5
:1050500068745365742E6E302E76616C3D2564FF46
:10506000FFFF00005765696768745365742E6E31E1
:105070002E76616C3D2564FFFFFF000004000020D8
:1050800043616C6962726174696F6E2E74382E743C
:1050900078743D2225332E346622FFFFFF00000086
:1050A0005BA16348FBF750F96148FBF7B6FAC0B261
:1050B000014607905E48FCF779FF4FF496715D4812
:1050C000006800F045FF5C48007805287ED15B4809
:1050D000806902465AA107905548FBF735F95448B4
:1050E000FBF79BFAC0B2014607905148FCF75EFF00
:1050F0005248007F08B1012000E00020024656A17E
:1051000007904B48FBF720F94948FBF786FAC0B2F5
:10511000014607904648FCF749FF4848407F08B1E0
:10512000012000E00020024651A107904048FBF713
:105130000BF93F48FBF771FAC0B2014607903C48B3
:10514000FCF734FF3D48807F08B1012000E00020DB
:1051500002464DA107903648FBF7F6F83448FBF7B6
:105160005CFAC0B2014607903148FCF71FFF334A92
:1051700020324BA12E48FBF7E7F82D48FBF74DFAFC
:10518000C0B2014607902A48FCF710FF2B4A403274
:1051900049A12748FBF7D8F82548FBF73EFAC0B2EB
:1051A000014607902248FCF701FF244A603248A1DB
:1051B0001F48FBF7C9F81E48FBF72FFAC0B201469B
:1051C00007901B48FCF7F2FE1C4A00E013E0803217
:1051D00045A11748FBF7B8F81548FBF71EFAC0B20F
:1051E000014607901248FCF7E1FE4FF49671114812
:1051F000006800F0ADFE1048007806287EF444AF49
:105200004FF496710B48006800F0A2FEFEF73CBF19
:1052100043616C6962726174696F6E2E74362E74AC
:1052200078743D2225332E306622FFFFFF000000F8
:1052300000120020B000002084000020B0010020F7
:105240005072696E742E6362302E7478743D22251C
:105250006422FFFFFF0000005072696E742E6274BA
:10526000302E76616C3D2564FFFFFF0000000000DA
:105270005072696E742E6274312E76616C3D2564B5
:10528000FFFFFF00000000005072696E742E627410
:10529000322E76616C3D2564FFFFFF0000000000A8
:1052A0005072696E742E74352E7478743D22257395
:1052B00022FFFFFF000000005072696E742E7436EA
:1052C0002E7478743D22257322FFFFFF000000003A
:1052D0005072696E742E74372E7478743D22257363
:1052E00022FFFFFF000000005072696E742E7438B8
:1052F0002E7478743D22257322FFFFFF000000000A
:1053000010B50021014800F02FFE10BD787C000888
:1053100010B504461CB902200649087008E005488B
:105320000078012804D0012002490870FEF75CFCD7
:1053300010BD00005C00002029B1064A92690243BA
:10534000044B9A6104E0034A92698243014B9A61DB
:10535000704700000010024000B587B0012108032B
:10536000FFF7EAFF01210420FFF7E6FFE020ADF898
:10537000180018208DF81B0003208DF81A0006A9CC
:105380001448FEF71FFA0020ADF804004FF48270B5
:10539000ADF806000020ADF808000220ADF80A00C4
:1053A0000120ADF80C004002ADF80E003820ADF839
:1053B00010000020ADF812000720ADF8140001A97C
:1053C000054800F041F80121034800F023F807B038
:1053D00000BD0000000801400030014010B5044647
:1053E00000BF02210A4800F021F80028F9D0214628
:1053F000074800F027F800BF0121054800F016F823
:105400000028F9D0024800F01AF8C0B210BD000020
:105410000030014021B1028842F04002028004E0E5
:1054200002884FF6BF731A40028070470246002080
:1054300013890B400BB1012000E0002070470146AA
:10544000888970478181704710B50022028802F474
:1054500041520B884C8823438C882343CC882343B8
:105460000C8923434C8923438C892343CC892343D0
:105470001A430280838B4FF2FF74234083830B8A8D
:10548000038210BD10B54FF480710448FEF76EFA28
:1054900008B1012010BD0020FCE700000008014019
:1054A00010B500F001F810BD0CB50020019000907F
:1054B0003348006840F480303149086000BF30480C
:1054C000006800F4003000900198401C01900098A2
:1054D00018B90198B0F5A06FF1D12948006800F41F
:1054E000003010B10120009001E0002000900098F1
:1054F000012843D12348006840F01000214908608A
:105500000846006820F0070008600846006840F080
:10551000020008601A484068194948600846406817
:1055200048600846406840F480604860084640682B
:1055300020F47C1048600846406840F4E810486059
:105540000846006840F08070086000BF0C480068A2
:1055500000F000700028F9D00948406820F00300EE
:10556000074948600846406840F00200486000BFB4
:105570000348406800F00C000828F9D10CBD000079
:10558000001002400020024010B51348006840F0AF
:1055900001001149086008464068104908400E495A
:1055A0004860084600680E4908400B4908600846F4
:1055B000006820F4802008600846406820F4FE005F
:1055C00048604FF41F008860FFF76AFF4FF00060EB
:1055D0000449086010BD0000001002400000FFF800
:1055E000FFFFF6FE08ED00E010B54FF08040008AA6
:1055F00020F001004FF0804108821848007860B325
:1056000017490888411C164A11800A2825D94FF0ED
:105610008040808920F001004FF080418881084659
:10562000008820F00100088000208884114608804E
:105630000A4908700B480078A5280ED10A4800785E
:10564000401E0849085CAA2807D10020064A1278A3
:1056500088540648006800F06FFC10BD72000020FE
:10566000700000204C010020730000207800002012
:10567000044900BF088800F020000028FAD088887C
:10568000C0B270470038014070B50546054C02E0D5
:10569000642000F0FDF9208800F080000028F7D099
:1056A000A58070BD0038014000B51F48008800F09B
:1056B000080038B11C4800881C4908701A48001DB1
:1056C000008848701848008800F0200058B3184837
:1056D0000078C0B9002017490870012014490870EB
:1056E00000204FF080418884134908804FF08040AB
:1056F000808940F001004FF0804188810846008891
:1057000040F00100088000204FF0804188840A4961
:10571000088008490A780978491C064B1970034922
:105720005018FCF76BFC00BD003801404C01002014
:1057300072000020730000207000002070B5044645
:105740000D4600260FE014F8010B00F011F802E0FE
:10575000322000F09DF90548008800F04000002844
:10576000F6D0701CC6B2AE42EDDB70BD0044004006
:105770000146044800BF028802F08002002AFAD0E5
:10578000818070470044004010B50021044800F0BB
:10579000BDFB04490860FCF753FBFCF781FB10BD1F
:1057A000747C000878000020F0B503460024002631
:1057B0000025002040F66A17B94200D100BF184604
:1057C000C1F3421401F01F06012707FA06F5012C68
:1057D00001D10C3004E0022C01D1103000E0143073
:1057E0001AB107682F43076002E00768AF430760FC
:1057F000F0BD00002DE9F04104462746F84300F0D3
:10580000FF08454645EA072500201D4908604FF47A
:10581000967000F03DF9102622E00020194908603A
:10582000642000F035F905F4004020B1012015494D
:10583000091D086003E000201249091D08604FF4AB
:10584000967000F025F94FF6FF7000EA450501203B
:105850000C4908604FF4967000F01AF9701EC6B239
:10586000002EDAD101200749091D08600649C1F858
:1058700098014FF4967000F00BF9BDE8F08100003C
:10588000B0012142988121420080214208B50121C6
:105890000420FFF751FD4FF400411B48FEF76FF85D
:1058A0004FF40040ADF8000003208DF802001020F6
:1058B0008DF8030069461448FDF784FF0121082094
:1058C000FFF73AFDC020ADF8000003208DF802007C
:1058D00014208DF8030069460C48FDF773FF012082
:1058E0000B4908600B49C1F89C010003ADF80000AA
:1058F00003208DF8020014208DF803006946024849
:10590000FDF760FF08BD000000080140000C0140E9
:105910009881214200802142490050EAC12018BFED
:1059200004204A0D18BF40F0010040F2FF72B2EBB4
:10593000515F08BF40F00200012808BF05207047F2
:1059400000280DDB00BF00BF00F01F0201219140C5
:105950004209920002F1E022C2F8001100BF00BF2C
:10596000704710B5002A06DA22F00042D21D22F05C
:105970000703102203E0D21C22F003030C2213B110
:105980009C188C4201D9012010BD0244014483605F
:10599000C0E90021C91AD018884202D81060024616
:1059A000F9E70020106010BD30380A2801D201202C
:1059B000704700207047000005490978002905D08C
:1059C00000684FF6FF71DFF80CC000DF7047000081
:1059D000E9000020F965000804490978002903D08E
:1059E0000068DFF80CC000DF70470000E90000200D
:1059F00021650008FFF74AFF00BF0A4800880A49EE
:105A00000988884209D007490888FBF709FE074939
:105A1000088004480088044908804FF4967000F01C
:105A2000E7F9EAE7380000204800002040000020A5
:105A300008480068C0010BD507480068C00707D0B8
:105A4000054880380068002802DA044901200870FF
:105A500070470000FCED00E0800E00E00C0100202B
:105A60004FF06042D36F002BFCD0036BD367D36F32
:105A7000002BFCD0C07840EA0120A2F87C007047DF
:105A80004FF06041CA6F002AFCD081F87C0070475B
:105A90003CE000BF00BF00BF00BF00BF00BF00BFB1
:105AA00000BF00BF00BF00BF00BF00BF00BF00BFFE
:105AB00000BF00BF00BF00BF00BF00BF00BF00BFEE
:105AC00000BF00BF00BF00BF00BF00BF00BF00BFDE
:105AD00000BF00BF00BF00BF00BF00BF00BF00BFCE
:105AE00000BF00BF00BF00BF00BF00BF00BF00BFBE
:105AF00000BF00BF00BF00BF00BF00BF00BF00BFAE
:105B000000BF00BF00BF00BF00BF00BF401EC0D22B
:105B1000704770B50D46040003D012B920780128F3
:105B200001D0802070BD204600F046FC28B12946F7
:105B3000204600F018F8002070BD812070BD10B51F
:105B400000F0B8FB10B10178022901D0802010BD0F
:105B50004188A1F57F42FF3A03D000F00BF8002006
:105B600010BD812010BD10B500F0D0FDBDE8104083
:105B700000F0BCBD10B5002100F0C8FDBDE810402C
:105B800000F0B4BD10B5029C016042608360C46047
:105B900010BD10B5029C016042608360C46010BDFE
:105BA0002DE9F04704460D462668D4E9010101F0CD
:105BB000C1FC80464046E16801F0BCFC074639461E
:105BC000404601F025FD20613146284601F0BAFF2C
:105BD0008146216901F0AEFE0746314601F0AAFC7C
:105BE00020604FF07E50216901F0ACFF074641462E
:105BF00001F0A0FE6060BDE8F0872DE9F0470446A3
:105C00000D462668D4E9010101F094FC8046404627
:105C1000E16801F08FFC07463946404601F0F8FC88
:105C200020613146284601F08DFF8146216901F04F
:105C300081FE0746314601F07DFC20604FF07E502A
:105C4000216901F07FFF0746414601F073FE606065
:105C5000BDE8F08701210920FFF76EFB01215848BC
:105C6000FDF73CFEFDF798FDFBF7FCFCFEF75CF949
:105C7000FDF73CFD4FF47A7000F0BAF8FBF7FAFC40
:105C80005048006801F0BAFD4F498860FEF7ECF813
:105C90000A287CD2DFE800F07B05121F2C3946531E
:105CA000606E32204949087049484A4908604A48AC
:105CB0004A490860B4204A49087075E05A204349AF
:105CC0000870484843490860474844490860B42080
:105CD0004349087068E064203C49087043483D49E6
:105CE000086041483D490860B4203D4908705BE0C8
:105CF00032203649087036483649086036483749F8
:105D00000860C820364908704EE064202F490870AA
:105D1000344830490860344830490860C820304968
:105D2000087041E0C82029490870304829490860B6
:105D30002D482A490860C8202949087034E0782095
:105D400022490870224823490860274823490860EF
:105D5000B4202349087027E078201C4908702148A6
:105D60001C49086020481D490860B4201C4908707F
:105D70001AE00CE07820154908701C4815490860A5
:105D8000194816490860B420154908700CE0002035
:105D90000E4908700E480F4908600F480F49086007
:105DA00000200F49087000BF00BFFFF7EDFCFDF7B2
:105DB000EBFD03E04FF47A7000F01AF8FAE7000008
:105DC000000230000800002028010020850000208B
:105DD0000AD7A33B880000200AD7A33C8C000020F0
:105DE000860000206F12033B0AD7233C6F12833AD0
:105DF000EFF3058109B182207047DFF808C000DFAA
:105E000070470000ED6D0008EFF3058008B18220B7
:105E10007047EFF31480C00703D0DFF80CC000DF39
:105E2000704700F0EDBF0000016E000888B0EFF38E
:105E3000058010B1822008B07047EFF3148010F095
:105E40000301134806D001291BD0022911D00329D0
:105E500019D113E008A981F309880078C0070BD095
:105E60005FF0020080F31488BFF34F8FBFF36F8F92
:105E700009E00078C00706D10320F3E70078C007E7
:105E800001D0FF20D7E7DFF80CC000DFD3E7000028
:105E90007C7D0008716E0008EFF3058008B10020DA
:105EA0007047DFF808C000DF70470000B96E0008D7
:105EB000EFF3058109B100207047EFF31481C907A2
:105EC00002D10449497819B1DFF80CC000DF7047EE
:105ED00001F020B8E8000020156F0008EFF30581FD
:105EE00009B182207047DFF808C000DF704700006A
:105EF000316F0008EFF305820AB182207047DFF8A6
:105F000008C000DF70470000536F0008EFF3058200
:105F10000AB100207047EFF31482D20702D1044A7D
:105F200052781AB1DFF80CC000DF704701F02EB8CC
:105F3000E80000208D6F0008EFF3058109B1FFF73D
:105F4000FEBDDFF808C000DF70470000B16F000839
:105F5000EFF3058212B14FF0FF307047DFF804C055
:105F600000DF7047D96F0008EFF305820AB1002007
:105F70007047EFF31482D20702D1044A52781AB163
:105F8000DFF80CC000DF704701F040B8E8000020E7
:105F90000D700008DFF80CC000DFDFF80CC000DF78
:105FA000FEE700007970000895700008EFF30580A7
:105FB00008B100207047DFF808C000DF704700001C
:105FC00079700008EFF3058109B182207047DFF88E
:105FD00008C000DF7047000095700008012806D057
:105FE000022805D0032804D0042804D102E003E0ED
:105FF00002E001E000E000BF00BF00BFFEE700BF1D
:10600000FEE70000074801684FF0E02041610021F1
:106010008161072101610448016841F07F4101600D
:1060200040177047787D000820ED00E070470000C1
:1060300002480068C0F380607047000004ED00E093
:106040004FF0E020806902490968081A7047000093
:10605000787D000850E8001F31B10B6840E800323D
:10606000002AF7D108467047BFF32F8FFAE710B523
:1060700068B161B10B3121F00302016844680B1A69
:106080001B1B934205D2084609680029F5D1002060
:1060900010BD210007D021180368C1E9003201605A
:1060A00001F1080010BD4260083010BD70B50D460A
:1060B000002812D04FF6FF71084C884204D22268A3
:1060C0000146104600F050FB20684570044800F07F
:1060D000DDF8BDE8704000F047BC70BDF000002066
:1060E000480300200F4810B50D4942680E480B6860
:1060F0000068934204D00A60CB88421E1A448A800A
:106100008A8880B282420AD100200860054800F0E7
:10611000BDF80146BDE81040024800F049BB10BD83
:1061200004010020480300200001002070B5194D33
:10613000E86800282CD0A88A401EA882002621E00A
:10614000A06838B161684160606810B1A168816081
:106150006660A6600F482146183800F029FBA08A27
:10616000A8826078042804D10B49E08A0988084491
:10617000A08201206070E068E860E06808B1056115
:10618000E6602661A88A002802D1EC68002CD7D1ED
:1061900070BD0000600300200001002070B5040005
:1061A0000FD00D4DA17801262868827891420CD934
:1061B00000F01AFB286846702046BDE8704000F0E9
:1061C000D3BB064800F062F8F7E766702146BDE8E9
:1061D0007040024800F0ECBAF000002048030020B4
:1061E0000321FFF763BF000010B50446008B08438E
:1061F00020836278618B062A18D0052A19D10842BB
:1062000017D001EA0002628388432083204600F011
:1062100016FB01206070628B0821204600F00BFB0A
:106220002146BDE81040034800F0C2BA31EA00023E
:10623000EAD010BD48030020814202D342688A425E
:1062400001D80120704702680A60BFF35F8F50E8F1
:10625000003F0A689A42F6D140E80012002AF2D1C3
:106260000020704768B161B10022083902E002469F
:10627000006830B18842FAD12AB10068106000206D
:1062800070470120704700214160F8E701464068EF
:1062900042684A600B780022022B05D0012B03D004
:1062A000032B01D04260704743680BB19960426094
:1062B00082607047810700D00020704770B50446A7
:1062C00000201546207001226270A17084F824100D
:1062D0006060A060E06020612062A082E082208394
:1062E000608384F82500E08C18B90548FFF7B2FEFA
:1062F000E06229462046BDE8704000F01DB800006D
:10630000B014002008B1082901D2012070470144CF
:10631000091F002201600A604260104670470000B9
:1063200003480021016003490988C18070470000CB
:10633000040100206C7D000870B5C28C1C4D9308D0
:1063400002D12A88C2F38D03C26A02EB830254078A
:1063500000D5121F4FF0807442E902140024264633
:10636000B2F1400242F82460641C0E2CFAD3C469D6
:106370001462826201632968C90014D5112B12D9F5
:106380004FF0FF31103B11EB53014FF0CC3305D0F0
:1063900042F8043C42F8083D491EF9D1C16A121F77
:1063A0008A4200D91360C06A0249016070BD0000D2
:1063B000687D0008A52E5AE2C1898089081A7047B5
:1063C000012202700022427082704260028142818A
:1063D000103982818908C181704700002DE9F041A0
:1063E000044640680E464FF0000804F10C05E8B37F
:1063F0006078012701283ED0022813D003285CD101
:106400000846FFF727FE050057D02046FFF73EFF5E
:106410000446294600F00CFA6770204600F00FFA97
:10642000214621E02046FFF731FF0646002100F01B
:10643000FFF92189F06904EB81010861D5E85F0F5C
:10644000401C81B2C5E8501F0028F7D12089401CAC
:1064500080B22081E189884201D1A4F80880777058
:10646000304600F0ECF93146174800E00CE0BDE89A
:10647000F04100F09DB92046FFF708FF0446324680
:10648000102100F0D8F9C7E7A089E189884216D227
:10649000208904EB80000661D5E85F0F401C81B2C3
:1064A000C5E8501F0028F7D12089401C80B2208108
:1064B000E189884201D1A4F80880BDE8F081BDE8F7
:1064C000F0410320FFF78ABD48030020002814D0C4
:1064D000411C13D00C4A4FF6FE7190420CD800EBD1
:1064E0004002C2EBC0120948036803EBC202521E0D
:1064F000B2FBF3F0884204D9084670474FF6FF70AC
:10650000704780B27047000000093D00887D000898
:10651000032101700021418041608160C1607047AA
:106520002DE9F0410446408820B1314DA1682A6828
:10653000914202D0FF20BDE8F081401E0004000C13
:10654000608053D12968086AA04209D1E0680862D6
:1065500008E0C268A24202D1E268C26002E01046CE
:106560000028F6D191F824000A6A06E053681BB1AE
:106570009B78834200D91846D268002AF6D18870E9
:10658000DFF870806168012611B32046FFF77EFEB8
:106590000746002100F04CF9384600F050F96680BB
:1065A000A760386AE0603C622968D8F804008A78FD
:1065B0008078824201D3384616E00E4800F0F8F8A1
:1065C00039460C4800F0F4F8286846707E700AE0FE
:1065D000D8F804108A782968824207D9054800F063
:1065E000E7F8286846700020FFF7D8FD0020A2E7F2
:1065F000F00000204803002070B51C4D0E460446F4
:106600004188286861B1A268824210D1A1F57F401B
:10661000FF3803D0491C6180002070BDFF2070BD91
:10662000A060016AE160046201206080F4E776B155
:1066300091788078814203D29070A06800F0DEF8F3
:10664000606830B12046296800F0B2F808E0012007
:1066500070BD2868606029680020486028688460F0
:1066600009213046FFF722FDF1E70000F00000208D
:1066700070B51B48012102685170006800F0B4F841
:10668000184D6C7818E000BF05EBC401486802782B
:10669000EAB1012A20D000F005F9E878641C8442B0
:1066A00000D100240F48801CD0E84F1F491EC9B2FA
:1066B000C0E8421F002AF7D1A8780028E4D16C7006
:1066C0000948FFF7E3FDBDE8704000F04DB90989C6
:1066D00089B2FFF789FDE0E78968FFF77FFEDCE715
:1066E000F0000020E0440020480300200548017825
:1066F00011B101214170704703494FF0805008608B
:1067000070470000F800002004ED00E0F0B4154DE3
:10671000AB1CEE784FEA0507D3E84F2FB24202D107
:10672000BFF32F8F11E0521CD4B2C3E8424F002AAE
:10673000F2D100BFD7E84F2F541CB44200D100243F
:10674000E4B2C7E8434F002BF4D1EB78934205D96C
:1067500005EBC202C2E90101F0BC7047F0BC0220A7
:10676000FFF73CBCE0440020104A10B5D368ABB141
:1067700013469B8A03E08CB12246A48A2344D46842
:106780008B42F8D3C460D0600261C46804B1206158
:10679000591A8182908A401A908210BD0024C460E8
:1067A000D060C91A02619182848210BD600300200A
:1067B00030B502780023022A03D0012A01D0032A2F
:1067C00000D101238C7800E01046426812B1957820
:1067D000A542F9D24A6041601BB102B19160886064
:1067E00030BD0020FBE7000003494A6842600022F8
:1067F00082604860704700004803002010B583683D
:1068000004462BB9607801280ED1084B03E09B6841
:1068100018780028FBD0204600F026F82146BDE875
:1068200010401846FFF7C4BF10BD00004803002009
:10683000806A01627047806AC0E90812704710B52B
:10684000016900290ED0C268CA60C36800223BB14A
:106850008B8A848A23448B82C3681961C26000E0FA
:106860008A82026110BD0000816839B142684A60C5
:106870004168002901D0806888607047054906E0BA
:106880004A68824202D14068486070471146002938
:10689000F6D17047480300200222027000224260B5
:1068A0004180704710B5416881B1FFF7EFFC0446A5
:1068B000FFF7C5FF0120607001462046FFF7B8FFD3
:1068C0002146BDE810400348FFF772BF4188491CCC
:1068D000418010BD4803002010B5416861B1FFF749
:1068E000D5FC04460121FFF7A3FF2046FFF7A7FFD1
:1068F0002046FFF753FC02E04188491C41800020FC
:1069000010BD000010B50C46418819B1491E4180E8
:10691000002010BD34B10A4A4368116823B1FFF763
:1069200047FF07E0012010BD416013680021596056
:106930001168886007212046FFF7B8FBF2E70000E6
:10694000F000002006480068D0E90A10814203D315
:1069500000680449884202D00120FFF73FBB70471E
:10696000F0000020A52E5AE207490222486042703A
:10697000064A1278002A05D006C98A4202D0C07899
:10698000FFF77EB870470000F00000200C010020E7
:1069900070B5FFF74DF800200446204A204902E078
:1069A00042F82040401C0B889842F9D31D483422FD
:1069B00001881D48FEF7D5FF1C48008880B240F0D2
:1069C00000421B4801681B48FEF7CBFF1A4808220B
:1069D00001881A480068FEF7C4FF194DFF20194AC4
:1069E000E870EC8400212846FFF768FC1648042173
:1069F0000170446015480170C460046184821448C9
:106A000015490560022068701248047044700978C6
:106A1000C170BDE87040FFF783BC000064450020F2
:106A2000647D0008907D000898120020687D0008B1
:106A3000947D0008B0140020B87D0008CC00002030
:106A400014030020FF5F00084803002060030020BB
:106A5000F0000020E04400209C7D00081B4810B599
:106A6000016841F47F01016000684FF07F4101EA55
:106A700000201649C0431439B0FA80F00968C0F10B
:106A80000800C1F30221814200D3481C0F49091FAD
:106A90000B686FF08072824063F317020A60FFF7A1
:106AA000B1FA0B49002808600EDB00F1E021FF225B
:106AB00081F8002400F01F0201219140400980006C
:106AC00000F1E020C0F8001110BD000020ED00E052
:106AD000FC0000200C4810B50268012151700068CC
:106AE000FFF782FEFFF7FEFA08480168491C0160C3
:106AF000FFF71CFB00F0EAFA0548FFF7C7FBBDE80B
:106B00001040FFF731BF0000F0000020000100201E
:106B100048030020002805D0810702D10178002910
:106B200000D000207047000030B50B4C0023626895
:106B300005E095688D4204D813461268491B002A67
:106B4000F7D10260816012B19568691A91600BB14A
:106B5000186030BD606030BDE80000202DE9F041D4
:106B60001E46174680460D4611F0FF0F00D14D1C02
:106B70001848FFF76FFA041E16D0280AE762E0846F
:106B8000E9B242462046E661FFF798FB012512482C
:106B9000124905E000EB850252F8042C32B16D1C5D
:106BA0000A889542F6D90020BDE8F081002DFAD080
:106BB00000EB850040F8044C0948E570007818B1F6
:106BC00001212046FEF74CFF2046FFF7E7FA284652
:106BD000EAE700009812002064450020647D000868
:106BE0000C0100202DE9F05F584DDFF85891DFF8D7
:106BF000588129684FF0010A002618B1CA78AB46BF
:106C0000824243D14E70F9F7E6FA29688862FFF7AD
:106C100099FE2868046A1FE06068C0B12046FFF74B
:106C200035FB07460021FFF703FE3846FFF707FE56
:106C300087F801A039464648FFF7BAFDE168A4F895
:106C400002A0A760386AE0603C620C4604E0E0689D
:106C50006680A660E6600446002CDDD12868C27814
:106C600008EB820141F8046CC16A3A48FFF7E4FA84
:106C70002868C66299F8001011B10021FEF7F0FEF5
:106C800035482968FFF7D8FA2E6056E0334909885D
:106C900088420CD808EB800858F8045C3DB12846BF
:106CA000FFF7E2FD2846FFF7CAFD2C6A22E0FF202D
:106CB000BDE8F09F6068C0B12046FFF7E7FA0746DD
:106CC0000021FFF7B5FD3846FFF7B9FD87F801A0B1
:106CD00039461F48FFF76CFDE168A4F802A0A760E1
:106CE000386AE0603C620C4604E0E0686680A660BA
:106CF000E6600446002CDDD148F8046C1548E96ACA
:106D0000FFF79AFAEE6299F8000018B100212846C0
:106D1000FEF7A6FE29461048FFF78EFA0C48DBF86E
:106D2000001040688B7882789A4209D981F801A0D6
:106D30000748DBF80010FFF73BFD0020FFF72EFAB5
:106D40000020B5E70C01002064450020F000002081
:106D500048030020B014002098120020647D000831
:106D600070B51A4D80B11A4A128890421FD8194A3C
:106D700002EB800050F8044CCCB1A17084F82410D0
:106D80002868A04205D014E028688170286880F83F
:106D90002410114840688078884215D90E48296827
:106DA000FFF706FD29680120487000200AE0FF2057
:106DB00070BD2046FFF722FD6078012804D1064807
:106DC000FFF764FAFFF7EAF9002070BDF000002039
:106DD000647D0008644500204803002002480068E4
:106DE000002800D0C0787047F000002010B50028BF
:106DF00004D0FFF76BFBFFF7F3F9402010BD000054
:106E000010B5134C207860B91248400705D11248DC
:106E100001681048FFF776FA08B1852010BDFFF72A
:106E2000B7FD0E49FF2009688870207858B9002105
:106E30000B4800F05DF80B49086000210A4800F09B
:106E4000E5F80A490860012020700020607010BD3C
:106E5000E8000020C0380020987D0008F0000020E5
:106E6000B07D0008C4000020A07D0008C000002004
:106E700070B50F4D687808B1002070BD0D4C2068CA
:106E800090F824100020FFF76BFF2068C178FF29DD
:106E900003D1816A203181F30988616811B960608A
:106EA00000202060FFF7DAFD01206870E4E70000B1
:106EB000E8000020F000002070B5FFF7C1F804469C
:106EC000FFF7B6F80849094E0D686D1C48B1FFF789
:106ED000B7F8A04200D204463068401C05FB0040D1
:106EE00070BD3068FAE70000787D000800010020DE
:106EF00010B5040005D0216819B1606808B10278A6
:106F00000AB1002010BD8900103189B2FFF758FA8C
:106F1000606810BD10B5002804D004680CB120785A
:106F200008B1002010BD2046FFF7F2FA204610BD40
:106F300010B5FFF7BFF910B10178032901D0802007
:106F400010BDFFF7EDFAFF2801D0002010BD812011
:106F500010BD70B50D46FFF7ADF9040002D02078E2
:106F6000032801D0802070BD2846FFF7AFFA014604
:106F70002046FFF741FB012803D0FF2804D0002062
:106F800070BD0DB1C12070BD812070BD10B500284D
:106F900007D0046824B1207810B9B1F5803F01DB37
:106FA000002010BD89B22046FFF776FC204610BDB8
:106FB00010B5FFF77FF910B10178022901D08020C8
:106FC00010BD4188A1F57F42FF3A03D0FFF784FC52
:106FD000002010BD812010BD70B50D46FFF76AF985
:106FE00004004FF0FF300DD0217802290AD1284645
:106FF000FFF76CFA01462046FFF784FC012802D017
:107000006088401C70BD002070BD000070B50E4649
:10701000040029D0206838B3606810F1030F23DB27
:10702000032821DCE16829B11048FFF720F80500AA
:107030001AD000E000256068E168001D40EA0121E7
:1070400033462A462068FFF789FD40B1084901EB25
:107050008000084950F8040C826A516370BD1DB16C
:1070600029460248FFF7FEF8002070BDC038002016
:1070700064450020955F000810B5FFF7AFFE0028BB
:1070800004D0034901EB800050F8040C10BD00004F
:107090006445002010B5FFF73DFD18B1C18C19B152
:1070A000C46A02E0802010BD0024C078FFF79AFD7A
:1070B000FF2806D01CB121460348FFF7D3F8002073
:1070C00010BD812010BD0000C03800202DE9F04126
:1070D000134E7468002C1CD0A068124F401E4FF055
:1070E0000108A06012E02546246874600022294649
:1070F0003868FEF70EFD10B10420FEF76FFF6879C7
:10710000012808D085F80480002C02D0A06800284F
:10711000E9D0BDE8F0812846E968FFF705FDF3E70F
:10712000E8000020C400002010B500290AD008782B
:10713000002807D005487844F9F78EFA002801D0D6
:10714000002010BD0248784410BD00005E0D000014
:10715000560D000021F00042A2F16052B2F5801FEE
:1071600001F0004328BFD2F17F6C0BD95FEA001C0D
:1071700043EAC20242EB507018BF704728BF20F0AC
:1071800001007047B2F5801FBCBF184670474FEA38
:10719000410C1CF5001F02D2084600F092BC70B5ED
:1071A00000F012F900000089FFF7F6BF4FF0004031
:1071B000A0F580007047491058BFC1F140415B10F5
:1071C00058BFC3F140438B42EFF30080704710F08B
:1071D000004248BF4042B0FA80F310FA03F10AD0EF
:1071E000C3F11D0303F580634FEA415002EB0352E4
:1071F00002EBD12170474FF00000704751EA030CB9
:1072000017D41CF5801F58BFBCF5801F00F1068005
:10721000994218BF704708BF9042704707D711F5D1
:10722000801F58BF13F5801F19D4994270478942B7
:1072300070471CF5801F08D5BCF5801FF7D58B4221
:1072400018BF704708BF824270474FF4001C1CEB08
:10725000410F38BF1CEB430F01D28B42704770B512
:1072600000F0B2F8922449004FF000514FF08053E3
:10727000FFF7A1BFDFF848C170B51CEA111E1EBFA1
:107280001CEA13159EEA0C0F95EA0C0F00F06F80B4
:1072900081EA030423EA4C134EEAD47E21EA4C111E
:1072A00041F4801143F48013AE44A1FB024CA0FBD7
:1072B0000365AEF17F7E361955EB0C05A1FB034C3F
:1072C0004CF10003A0FB021C16EB0C06654153F1C8
:1072D0000003094218BF46F0010613F4007F0BD1EA
:1072E0004FEA03314FEA0530340341EA155140EAD1
:1072F00016506FF003020AE04FEAC3214FEAC5209F
:10730000F40241EA555140EA56506FF0020202EB96
:107310002E4201EB025585EACE710AD05FEA440C99
:1073200018BF24F0004450F1000041F1000120EAB0
:10733000D47040F2FE7C624500D270BDA84214BFFA
:107340004FF080444FF04044002E08BF0024BEF1AF
:10735000806FA8BFA1F1C041BDE8704080F282807B
:107360004FF0000001F1C04101F0004170479EEA7A
:107370000C0F0CEA131518BF95EA0C0F06D04FF04E
:10738000000081EA030E0EF0004170BD00F01CF811
:107390008900013E00F007B800F009B84FEA430C3D
:1073A0005FEA5C5C08D081EA030100F05BB84FEA59
:1073B000410C5FEA5C5CF6D14FF000000149704778
:1073C0000000FF070000F87F0EF1020E2EF0030E02
:1073D0005EF8046B364205D4012A43EB030515F52C
:1073E000001F12D8012841EB010C1CF5001F0CD81E
:1073F0000ED14FEAD17C15F5001F0CEB4C0C0CF1B3
:10740000020C08BF4CEBD37C04E04FF0080C01E009
:107410004FEAD37C0CEB4C0526FA05F606F007067E
:10742000B6F1040C06D20EEB860CBDE870404CF0B1
:10743000010C6047DFE80CF0090B02024FF000413D
:107440004FF00000A1F5002170BD1946104601283B
:1074500051EB010418BFD4F5001484BF002001F0E3
:10746000004170BD0808A0F500114FEA31017047D6
:1074700053EA010C17D41CF5801F58BFBCF5801FC0
:1074800000F106808B4218BF704708BF82427047E8
:1074900007D713F5801F58BF11F5801F19D48B42F1
:1074A00070479B4270471CF5801F08D5BCF5801FB4
:1074B000F7D5994218BF704708BF904270474FF404
:1074C000001C1CEB430F38BF1CEB410F01D299424B
:1074D00070470FB40CBC03BCFFF7C1BE43004FEABA
:1074E000D30C4FEA3C0C43401FBF40070CF16051E6
:1074F00013F0FE4F70471CF0006F03D100200CF01A
:10750000004170470CF0004343EA507010B540EA68
:10751000CC0000F090FA00BF000000924FEA00019A
:10752000FFF7A0BF4FF000414FF00000A1F5002190
:107530007047000090EA010F48BF81F0004100F160
:107540000883421A3CBF801A89184FEAD0524FF084
:107550007F4C1CEA410FA2EBD15318BF9CEA026F8B
:1075600000F03B804FF0004C4CEA00204CEA012137
:1075700021FA03FC10EB0C0C1ED202F1FF325FEA81
:107580001C2040EBC25038BF70471CF07F0F4FEA01
:10759000400C18BFBCF17F4F38BF7047C3F12003C8
:1075A000994008BF20F00100BCF17F4F38BF704701
:1075B000A0F1C04000F085BA4FEA3C00000A40EB61
:1075C000C25028BF1CF0FF0F4FEA400CE6D018BF96
:1075D000BCF17F4F38BF7047EAE79CEA026F05D0E5
:1075E00010EA5C0F08BF00F00040704710B500F0D3
:1075F00022FA00BF64FBBE3E401058BFC0F14040BD
:10760000491058BFC1F140418142EFF300807047FB
:107610004FF47F0C1CEAD0121EBF1CEAD11392EA71
:107620000C0F93EA0C0F00F0858090EA010F48BF21
:1076300042F4807240F4000C41F400002CF07F41D1
:1076400020F07F4000B58142A2EB03020FF2081C3C
:10765000ACEB504EC0F100009EF800E04FEA4E0E39
:1076600000FB0EFC38BF49004FEA2C1C02F5FA0261
:107670000CFB0EF34FEACE1E4FEA112C4FEAC1214C
:107680000EEB635E42EB22420EFB0CFC4FEA1C53F6
:1076900000FB03114FEA112C4FEA01310EFB0CFCE9
:1076A0004FEADC4C00FB0C11C14228BF09184CEB1F
:1076B00003335DF804EB10EB410143EBC250B2F52C
:1076C0007C0F38BF704729D512F0F00F1CBF00F1B6
:1076D000C04000F000407047008182838485868727
:1076E00088898B8C8D8E8F919293959697999A9C81
:1076F0009D9FA0A2A3A5A7A8AAACAEB0B2B3B5B7F0
:10770000B9BCBEC0C2C5C7C9CCCED1D4D7D9DCDFC5
:10771000E2E6E9ECF0F3F7FAFE0000004FEA400C75
:107720000CF1807CBCF17E4F28BF7047B0F1C040A7
:1077300000F0C7B990EA010F0CEAD11348BF42F438
:107740008072624538BF634507D213F47F0F16D0AD
:1077500080EA010000F00040704710B500F06BF9BE
:10776000097EFC3E00F005B880EA010000F0004010
:10777000704780EA010000F0004000F0A2B912F466
:107780007F0F04BF0248704780EA010000F099B9FA
:107790000000C07F50EA010C00F113801CF5000FBF
:1077A00058BFBCF5000F01D48842704707D710F5C9
:1077B000000F58BF11F5000F15D488427047894259
:1077C00070471CF5000F04D5BCF5000FF7D58142BA
:1077D00070474FF0807C1CEB400F38BF1CEB410F13
:1077E00001D28142704710B500F025F9922449007A
:1077F0004FF000504FF08051FFF7FEBE41000B0EDE
:10780000D3F19E0208D950F400034FEA032323FA70
:1078100002F048BF4042704710B500F00CF900BFBD
:1078200049922480002070476FF0004282EA2000D5
:1078300070470000C10DD1F19E0206DB4FEA002324
:1078400043F0004323FA02F07047004207D54FEAA5
:107850004001B1F1FE4F02D24FF00000704710B569
:1078600000F0E9F849922480002070476FEA200078
:107870007047000010F0004148BF4042B0FA80F36A
:1078800010FA03F2C3F19D030BD051EAC35101EB8F
:107890001220530638BF704700F1010008BF20F0E6
:1078A00001007047B0FA80F310FA03F2C3F19D03B0
:1078B0000AD0D90501EB1220530638BF704700F1FA
:1078C000010008BF20F001007047000050EA010CE1
:1078D00000F113801CF5000F58BFBCF5000F01D458
:1078E0008842704707D710F5000F58BF11F5000FF9
:1078F00015D488427047894270471CF5000F04D5A3
:10790000BCF5000FF7D5814270474FF0807C1CEB2F
:10791000400F38BF1CEB410F01D28142704710B5B8
:1079200000F089F8922449004FF000504FF0805148
:10793000FFF762BE4FF47F0C1CEAD0121EBF1CEA98
:10794000D11392EA0C0F93EA0C0F00F0478090EAF3
:10795000010F48BF42F480724FF0004C4CEA002007
:107960004CEA012102EB0302A0FB0113A2F5000285
:10797000002918BF43F001035B0028BF4FEA33031F
:1079800042EB22425FEA132C4CEBC2502EBFBCEB01
:10799000436FB2F57C0F70474FEA036CBCF1004FA8
:1079A00008BF20F00100B2F57C0F38BF70470BD53F
:1079B00082F0FF0212F5803FC8BF704700F1C0405F
:1079C000D8BF00F00040704700F5000C5FEA4C0C97
:1079D00048BF7047B0F1C04000F073B890EA010FA3
:1079E0000CEAD11348BF42F48072624538BF634548
:1079F00004D280EA010000F00040704710B500F0AA
:107A00001AF800BF8900013E00F007B800F009B87D
:107A10005FEA410C5FEA1C6C08D080EA010000F0CC
:107A200050B85FEA400C5FEA1C6CF6D14FF00040A2
:107A3000A0F5800070470EF1020E2EF0030E5EF8E6
:107A4000044B244204D44FEA4102B2F17F4F11D8D3
:107A50004FEA4003B3F17F4F0CD80ED14FEAD07CF0
:107A6000B2F17F4F0CEB4C0C0CF1020C08BF4CEB4D
:107A7000D17C04E04FF0080C01E04FEAD17C0CEB24
:107A80004C0324FA03F404F00704B4F1040C06D206
:107A90000EEB840CBDE810404CF0010C6047DFE8B1
:107AA0000CF0070802024FF00040A0F5800010BD66
:107AB0000846420018BFD2F1807288BF00F0004033
:107AC00010BDFF2141EAD050C005704751EA000CBB
:107AD00000F113801CF5000F58BFBCF5000F01D456
:107AE0008142704707D711F5000F58BF10F5000FFE
:107AF00015D481427047894270471CF5000F04D5A8
:107B0000BCF5000FF7D5884270474FF0807C1CEB26
:107B1000410F38BF1CEB400F01D28842704780EA0A
:107B2000010081EA000180EA0100FFF7F8BE80F061
:107B3000004090EA010F7FF504AD81F0004100F0B4
:107B400008B8000090EA010F48BF81F000413FF5FE
:107B5000F8AC421A04D882F00042A0EB02001144B3
:107B60004FEAD0524FF07F4C1CEA410FA2EBD153A9
:107B700018BF9CEA026F4AD04FF0004C4CEA00203C
:107B80004CEA012121FA03FCB0EB0C0C0FD412F0EB
:107B9000FE0F36D05FEA4C001DD5001240EBC250FC
:107BA00038BF70471CF03F0F18BF70470BE0A2F1C1
:107BB00001025FEA1C2040EBC25038BF70471CF046
:107BC0007F0F18BF7047C3F12003994014BF401EB8
:107BD00020F00100704780084FEA122308BF704769
:107BE000B0FA80FCA2EB0C02CCF1280C60FA0CF08D
:107BF00093EA122F04BF00EBC25070474FEAC370E4
:107C00007047130A5FEADC1008BF7047F6E79CEA8A
:107C1000026F04D010EA5C0F08BF0020704710B557
:107C2000FFF709FF40DFF63E81F000407047F8F7AC
:107C300088BE0000D5180008000000000100000008
:107C400000000000F55900080000000001000000DD
:107C500000000000F93B00080200000001000000E5
:107C600000000000A93E0008000000000100000024
:107C7000000000007C000020E93F00080000000038
:107C800001000000000000000920000800000000C2
:107C900001000000000000002020D1F9C6B7C3FB9E
:107CA000A3BA25730D0A2020B2E2CAD4CAB1BCE43B
:107CB000A3BA25730D0A2020C6F0CABCD6D8C1BF0E
:107CC000A3BA252E3366670D0A2020BDE1CAF8D677
:107CD000D8C1BF3A20252E3366670D0A2020BAACE2
:107CE000CBAEC1BF3A20252E32662525200D0A20B5
:107CF00020BAACB9CCC1BF3A20252E326625250D5D
:107D00000A2000002020D1F9C6B7C3FBA3BA25730F
:107D10000D0A2020B2E2CAD4CAB1BCE4A3BA2573CA
:107D20000D0A2020C6F0CABCD6D8C1BFA3BA25739D
:107D30000D0A2020BDE1CAF8D6D8C1BF3A2025736C
:107D40000D0A2020BAACCBAEC1BF3A202573200D5E
:107D50000A2020BAACB9CCC1BF3A2025730D0A2045
:107D6000000000000A0000000004020105000100FC
:107D700000A24A04480000003F1901000100000071
:107D80000200010052000400E803000000000000AF
:107D90001402000010240000200C0000100000005D
:107DA00000000000000000000000000000000000D3
:107DB000000000008C45002000000000555C000819
:107DC000000000000100000000080000040000089E
:107DD0000000000000000002000100001000000090
:107DE00002400000000000A000000000054000006C
:107DF000000000C8000000000C4000000000409C93
:107E000000000000194000000020BCBE000000007F
:107E100034400000BFC91B8E00000004B5400000C4
:107E2000504BCFD06607E2CF010000006C4100004C
:107E30003E8251AADFEEA73401000000D9420000C3
:107E4000DCB5A0E23A301F97FFFFFFFFB44500000A
:107E5000FD25A0C8E9A3C14FFFFFFFFFFF3F0000C2
:107E60000000008000000000FF3F000000000080D4
:107E700000000000B07E000800000020100100009B
:107E800028010008C07F000810010020CC48000035
:107E9000440100081C00000043000000F8FFFFFF41
:107EA0000C0000000E0000000F0000002E0000007B
:107EB00000000000000000000000000000000000C2
:107EC00000000000000000000000000000000000B2
:107ED00000000000000000000000000000000000A2
:107EE0000000000000000000000000000000000092
:107EF0000000000000000000000000000000000082
:107F00000000000000000000000000000000000071
:107F1000000000000000803F0000000000000000A2
:107F20000000000000000000000000000000000051
:107F3000000000000D000000000000000000000034
:107F40000000000000000000000000000000000031
:107F500000000000000064000000000000000000BD
:107F60000000000000000000000000000000000011
:107F70000000000000000000000000000000000001
:107F80000000000000A24A04000000000000000001
:107F900001020304060708090000000000000000B9
:107FA00000000000000000000000000000000000D1
:107FB00000000000000000000000000000000000C1
:04000005080000ED02
:00000001FF
